:100000000C94D2030C94EF030C94822B0C94EF030A
:100010000C94EF030C94EF030C94EF030C94EF0398
:100020000C94EF030C9459420C94EF030C94EF03DF
:100030000C94EF030C94EF030C94EF030C94EF0378
:100040000C94EF030C94EF030C94EF030C94EF0368
:100050000C94EF030C94F0500C94EF030C94EF030A
:100060000C94EF030C94EF030C94EF030C94EF0348
:100070000C94EF030C94EF030C94EF030C94EF0338
:100080000C94EF030C94EF030C94EF030C94EF0328
:100090000C94EF03DE432944E8440E458645AA4507
:1000A000CF45D345E345584E584E584E584E584EBE
:1000B000584E584E584E584E584E584E584E584E10
:1000C000584E584E584E584E584E584E584E584E00
:1000D000584E7646F3450F469446A446184859486C
:1000E000DA481C495849CB49584E584E584E584E3C
:1000F000584E584E584E584E584E584E584E584ED0
:10010000584E584E584E584E584E584E584E584EBF
:10011000584ED3461847394A524A824A994A584E4D
:10012000584E584E584E584E584E584E584E584E9F
:10013000584E4847A047A64A264BA54BE74B9A4D39
:10014000A94D5E4C724CB84DCA4DDD4D584EEE4D2A
:100150008547AD47D547224E3D4E284C434C864CF3
:10016000BA4CDD4C294D444D6F4DCE03C103B30352
:10017000A30390037A036103470329030803E602FC
:10018000C2029E0276024F02280203026C01B801ED
:1001900096017501560139011F010601EF00DA00D1
:1001A000B5008200A5009600000043414E203100BA
:1001B00000000000000000000043414E203200001B
:1001C000000000000000000043414E20330000000A
:1001D0000000000000000043414E203400000000F9
:1001E00000000000000043414E20350000000000E8
:1001F000000000000043414E2036000000000000D7
:100200000000000043414E203700000000000000C5
:1002100000000043414E20380000000000000000B4
:10022000000043414E2039000000000000000000A3
:100230000043414E2031300000000000000000006B
:1002400043414E2031310000000000000000004317
:10025000414E203132000000000000000000434108
:100260004E20313300000000000000000043414EEA
:1002700020313400000000000000000043414E2007
:10028000313500000000000000000043414E2031E5
:100290003600000000000000000043414E203137CE
:1002A00000000000000000000043414E20313800F3
:1002B000000000000000000043414E2031390000E2
:1002C0000000000000000043414E203230000000DA
:1002D00000000000000043414E20323100000000C9
:1002E000000000000043414E2032320000000000B8
:1002F0000000000043414E203233000000000000A7
:1003000000000043414E2032340000000000000095
:10031000000043414E203235000000000000000084
:100320000043414E20323600000000000000000073
:1003300043414E203237000000000000000000431F
:10034000414E203238000000000000000000434110
:100350004E20323900000000000000000043414EF2
:1003600020333000000000000000000043414E2018
:10037000333100000000000000000043414E2033F4
:1003800032000000000000000000466C617368202D
:10039000310000000000000000466C6173682032EC
:1003A0000000000000000000466C6173682033000C
:1003B00000000000000000466C61736820340000FB
:1003C000000000000000466C6173682035000000EA
:1003D00000000000005357495443482031000000FA
:1003E00000000000535749544348203200000000E9
:1003F00000000053574954434820330000000000D8
:1004000000005357495443482034000000000000C6
:1004100000535749544348203500000000000000B5
:100420005357495443482036000000000000005351
:10043000574954434820370000000000000053573C
:100440004954434820380000000000000053574939
:10045000544348203900000000000000535749541D
:1004600043482031300000000000005357495443F6
:10047000482031310000000000004348414E4E4505
:100480004C20310000000000004348414E4E454CD6
:1004900020320000000000004348414E4E454C20F1
:1004A000330000000000004348414E4E454C2034CC
:1004B0000000000000004348414E4E454C203500EE
:1004C00000000000004348414E4E454C20360000DD
:1004D000000000004348414E4E454C2037000000CC
:1004E0000000004348414E4E454C203800000000BB
:1004F00000004348414E4E454C20390000000000AA
:10050000004348414E4E454C203130000000000071
:100510004348414E4E454C2031310000000000431D
:1005200048414E4E454C2031320000000000434807
:10053000414E4E454C2031330000000000434841FD
:100540004E4E454C20313400000000004348414EDF
:100550004E454C20313500000000004348414E4ECE
:10056000454C20313600000000004348414E4E45C6
:100570004C20313700000000004348414E4E454CAE
:1005800020313800000000004348414E4E454C20C9
:10059000313900000000004348414E4E454C2032A6
:1005A0003000000000004348414E4E454C2032319F
:1005B00000000000004348414E4E454C20323200BE
:1005C000000000004348414E4E454C2032330000AD
:1005D0000000004348414E4E454C2032340000009C
:1005E00000004348414E4E454C203235000000008B
:1005F000004348414E4E454C20323600000000007A
:100600004348414E4E454C20323700000000004325
:1006100048414E4E454C203238000000000043480F
:10062000414E4E454C203239000000000043484105
:100630004E4E454C20333000000000004348414EF0
:100640004E454C20333100000000004348414E4EDF
:10065000454C20333200000000004348414E4E45D7
:100660004C20333300000000004348414E4E454CBF
:1006700020333400000000005649525455414C20AC
:10068000310000000000005649525455414C2032C0
:100690000000000000005649525455414C203300E0
:1006A00000000000005649525455414C20340000CF
:1006B000000000005649525455414C2035000000BE
:1006C0000000005649525455414C203600000000AD
:1006D00000005649525455414C203700000000009C
:1006E000005649525455414C20380000000000008B
:1006F0005649525455414C20390000000000005624
:1007000049525455414C20313000000000005649F8
:10071000525455414C2031310000000000564952DE
:100720005455414C203132000000000056495254CB
:1007300055414C20313300000000005649525455B9
:10074000414C2031340000000000564952545541BC
:100750004C20313500000000005649525455414CA0
:1007600020313600000000005649525455414C20BB
:10077000313700000000005649525455414C203199
:100780003800000000005649525455414C20313980
:1007900000000000005649525455414C20323000B0
:1007A0000000000011241FBECFEFD0E1DEBFCDBF9F
:1007B00011E0A0E0B1E0ECE2F6EC00E00BBF02C01B
:1007C00007900D92AA3AB107D9F71EE0AAEAB1E064
:1007D00001C01D92A33FB107E1F70C9476350C944C
:1007E0000000282F277099279695879596958795CD
:1007F0009695879533272330310529F1243031052B
:100800004CF421303105B9F022303105C4F4232BEA
:1008100071F02CC025303105F1F025303105BCF0E8
:1008200026303105E1F027303105E9F01FC0A098EE
:10083000A198A2981BC0A09AA198A29817C0A098AE
:10084000A19AA29813C0A09AA19AA2980FC0A098AA
:10085000A198A29A0BC0A09AA198A29A07C0A098AA
:10086000A19AA29A03C0A09AA19AA29A80628093A8
:100870007C0080917A00806480937A0080917A0075
:1008800084FFFCCF80917A00806180937A00209170
:100890007800809179009927880F991F880F991FF8
:1008A0002295269526952370820F911D0895282F55
:1008B000277099279695879596958795969587950C
:1008C00033272330310529F1243031054CF4213010
:1008D0003105B9F022303105C4F4232B71F02CC05E
:1008E00025303105F1F025303105BCF026303105D9
:1008F000E1F027303105E9F01FC0A098A198A29837
:100900001BC0A09AA198A29817C0A098A19AA298DB
:1009100013C0A09AA19AA2980FC0A098A198A29AD9
:100920000BC0A09AA198A29A07C0A098A19AA29AD7
:1009300003C0A09AA19AA29A806280937C008091C1
:100940007A00806480937A0080917A0084FFFCCFE3
:1009500080917A00806180937A0080917900992754
:10096000089540E050E0FC01029625913491621711
:10097000730760F44B5F5F4FFC0102962591349141
:100980006217730718F446395105A4F3CA01089594
:10099000FC01809100018130B1F410920001F093CC
:1009A000B301E093B201F093B101E093B001F09391
:1009B000AF01E093AE01F093AD01E093AC01F09391
:1009C000AB01E093AA016091B0017091B101709305
:1009D000B3016093B2014091AE015091AF015093C9
:1009E000B1014093B0012091AC013091AD01309341
:1009F000AF012093AE018091AA019091AB01909339
:100A0000AD018093AC01F093AB01E093AA01E80F34
:100A1000F91FE20FF31FE40FF51FCF01860F971F99
:100A200065E070E00E945D62CB01089580E10E9464
:100A3000F1030E94C804BC018AE691E00E94B1045F
:100A40009927089583E10E9457049FE4899FC0017C
:100A50001124880F892F881F990B9195A82F8091B9
:100A600001018130C1F4109201018A2F99279093DE
:100A7000BD018093BC019093BB018093BA01909318
:100A8000B9018093B8019093B7018093B601909318
:100A9000B5018093B401E091BA01F091BB01F093EC
:100AA000BD01E093BC016091B8017091B9017093F0
:100AB000BB016093BA014091B6015091B7015093C8
:100AC000B9014093B8012091B4013091B501309340
:100AD000B7012093B6018A2F99279093B50180938F
:100AE000B401820F931F840F951F860F971F8E0FDF
:100AF0009F1F65E070E00E945D62862F9927089530
:100B000080E280937C0087E880937A00989A999A93
:100B10009A9AA098A198A298089590E0892F82951A
:100B2000807F8093ED001092EE001092EF00109203
:100B3000F0001092F1001092F2001092F300109267
:100B4000F4001092F5001092F6001092F70080E089
:100B50001092FA008F5F8830D8F39F5F9F30F0F2D9
:100B600008953091ED0090E020EC892F8295807FF0
:100B70008093ED008091EF00822329F43093ED0003
:100B8000892F992708959F5F9F3078F33093ED0068
:100B90008FEF90E008958091EE0086FF03C080E023
:100BA00090E008958091EE0085FF03C081E090E021
:100BB00008958091EF00807C19F48FEF90E0089504
:100BC00082E090E00895BC0140E08091EF00992719
:100BD0008F709070892B89F0FB01E40FF11D8091DB
:100BE000FA0080834F5F242F33278091EF009927ED
:100BF0008F709070281739077CF308958FE79DE078
:100C00000E94C33265E27EE080E00E9400336DED19
:100C10007DE081E00E94003367E97DE082E00E9490
:100C2000003381E08093BE0180917F0D813061F4BB
:100C30008091800D9091810D6AE070E00E945D626C
:100C400070937D0D60937C0D8091260E813061F450
:100C50008091270E9091280E6AE070E00E945D62FC
:100C60007093780D6093770D8091DE0D813061F483
:100C70008091DF0D9091E00D6AE070E00E945D626E
:100C800070937B0D60937A0D8091980D813061F4A3
:100C90008091990D90919A0D6AE070E00E945D62DA
:100CA0007093240E6093230E0895CF93DF93CDB7F6
:100CB000DEB7CE55D0400FB6F894DEBF0FBECDBF25
:100CC00019828CE0888F84E690E09B838A831D8262
:100CD0001C821E821F82188619861A861B868981AD
:100CE0009E01245F3F4FF901E80FF11D10828F5FD5
:100CF0008C30C8F3CE0101960E94B332A895198EAC
:100D00001A8E84E690E09C8F8B8F1E8E1D8E898DAF
:100D10009E012F5F3F4FF901E80FF11D168E8F5F87
:100D20008232C8F3CE0149960E94D332A89581E061
:100D3000898F1A8E84E690E09C8F8B8F1E8E1D8E7D
:100D40008A8D9E012F5F3F4FF901E80FF11D168E2E
:100D50008F5F8232C8F3CE0149960E94D332A895A4
:100D600082E0898F1A8E84E690E09C8F8B8F1E8E96
:100D70001D8E8A8D9E012F5F3F4FF901E80FF11DF7
:100D8000168E8F5F8034C8F3CE0149960E94D3320D
:100D9000C25ADF4F0FB6F894DEBF0FBECDBFDF9152
:100DA000CF91089599278832910509F440C089327E
:100DB000910594F48532910559F18632910534F408
:100DC00083329105D9F08497F1F04FC086329105B6
:100DD00021F1879739F149C08B329105B9F18C32F5
:100DE000910534F48932910539F18A9751F13DC06A
:100DF0008C32910581F18D9799F137C080EC0E947A
:100E000025419927089581EC0E942541992708954D
:100E100082EC0E9425419927089581ED0E94254189
:100E20009927089584EC0E9425419927089585EC1F
:100E30000E9425419927089586EC0E942541992713
:100E4000089587EC0E9425419927089583EC0E941C
:100E500025419927089582ED0E94254199270895FB
:100E600083ED0E9425419927089580E090E0089540
:100E7000EF92FF920F931F93CF93DF93CDB7DEB71F
:100E800065970FB6F894DEBF0FBECDBF8091750E8B
:100E90009091760E01978F5F974008F0ACC39091C8
:100EA000740E992309F4A7C38091790D8F5F809305
:100EB000790D891708F49FC31092790D88E08D830E
:100EC00080917E0D99278530910509F4AAC286305C
:100ED00091059CF48230910509F4FEC1833091059F
:100EE00024F4019709F4C1C117C08330910509F4B6
:100EF0002AC2049709F45EC20FC08730910509F435
:100F0000E7C2873091050CF4B8C28930910509F425
:100F10000CC30A9709F444C38091750E9091760E24
:100F2000AA27BB2789839A83AB83BC8301E0009304
:100F30007E0D10E080EC0E9425418111102F81EC84
:100F40000E9425418111126082EC0E94254181118D
:100F5000146081ED0E9425418111186084EC0E948B
:100F600025418111106185EC0E942541811110629B
:100F700086EC0E9425418111106487EC0E94254176
:100F8000811110681E8310E083EC0E9425418111BD
:100F900011E082ED0E9425418111126083ED0E94D3
:100FA0002541811114601F8310E081E090E00E94D0
:100FB0002654892B09F011E082E090E00E9426542B
:100FC000892B09F0126083E090E00E942654892B5F
:100FD00009F0146084E090E00E942654892B09F007
:100FE000186085E090E00E942654892B09F010617A
:100FF00086E090E00E942654892B09F0106287E079
:1010000090E00E942654892B09F0106488E090E05B
:101010000E942654892B09F01068188710E089E097
:1010200090E00E942654892B09F011E08AE090E0BC
:101030000E942654892B09F012608BE090E00E94F8
:101040002654892B09F014608CE090E00E9426540D
:10105000892B09F018608DE090E00E942654892BBE
:1010600009F010618EE090E00E942654892B09F06F
:1010700010628FE090E00E942654892B09F01064E2
:1010800080E190E00E942654892B09F010681987AE
:1010900010E081E090E00E94E710892B09F011E058
:1010A00082E090E00E94E710892B09F0126083E053
:1010B00090E00E94E710892B09F0146084E090E032
:1010C0000E94E710892B09F0186085E090E00E94EB
:1010D000E710892B09F0106186E090E00E94E7108C
:1010E000892B09F0106287E090E00E94E710892BBD
:1010F00009F0106488E090E00E94E710892B09F065
:1011000010681A8710E089E090E00E94E710892BB0
:1011100009F011E08AE090E00E94E710892B09F0C5
:1011200012608BE090E00E94E710892B09F01460B8
:101130008CE090E00E94E710892B09F018608DE0A8
:1011400090E00E94E710892B09F010618EE090E09A
:101150000E94E710892B09F010628FE090E00E9456
:10116000E710892B09F0106480E190E00E94E710FD
:10117000892B09F010681B8710E081E190E00E9444
:10118000E710892B09F011E082E190E00E94E7105E
:10119000892B09F0126083E190E00E94E710892B0F
:1011A00009F0146084E190E00E94E710892B09F0B7
:1011B000186085E190E00E94E710892B09F010612A
:1011C00086E190E00E94E710892B09F0106287E128
:1011D00090E00E94E710892B09F0106488E190E00C
:1011E0000E94E710892B09F010681C8710E089E144
:1011F00090E00E94E710892B09F011E08AE190E06D
:101200000E94E710892B09F012608BE190E00E94A8
:10121000E710892B09F014608CE190E00E94E71040
:10122000892B09F018608DE190E00E94E710892B6E
:1012300009F010618EE190E00E94E710892B09F01F
:1012400010628FE190E00E94E710892B09F0106492
:1012500080E290E00E94E710892B09F010681D875A
:10126000CE0101960E94463FC6C18091750E9091B5
:10127000760E0196AA27BB2789839A83AB83BC830A
:1012800082E080937E0D00E00F2EF6E0EF2EFF242B
:10129000F02DEC0EFD1E802F8F5F0E948C29FC012B
:1012A000878580FF02C014E60BC0878583FF02C0DC
:1012B00015E606C08181803F11F411E001C010E005
:1012C000F701E00FF11D10830F5F083020F3CE010E
:1012D00001960E94463F8FC18091750E9091760EC7
:1012E0000296AA27BB2789839A83AB83BC8383E0BA
:1012F00080937E0D00E00F2EF6E0EF2EFF24F02D00
:10130000EC0EFD1E802F875F0E948C29FC018785D3
:1013100080FF02C014E60BC0878583FF02C015E67C
:1013200006C08181803F11F411E001C010E0F70197
:10133000E00FF11D10830F5F083020F3CE010196FE
:101340000E94463F58C18091750E9091760E03968B
:10135000AA27BB2789839A83AB83BC8384E08093CD
:101360007E0D00E00F2EF6E0EF2EFF24F02DEC0EA8
:10137000FD1E802F8F5E0E948C29FC01878580FFD7
:1013800002C014E60BC0878583FF02C015E606C0C5
:101390008181803F11F411E001C010E0F701E00FFE
:1013A000F11D10830F5F083020F3CE0101960E94DB
:1013B000463F21C18091750E9091760E0496AA2722
:1013C000BB2789839A83AB83BC8385E080937E0DA2
:1013D00000E00F2EF6E0EF2EFF24F02DEC0EFD1EA8
:1013E000802F875E0E948C29FC01878580FF02C0C8
:1013F00014E60BC0878583FF02C015E606C0818115
:10140000803F11F411E001C010E0F701E00FF11D81
:1014100010830F5F083020F3CE0101960E94463FF3
:10142000EAC08091750E9091760E0596AA27BB278B
:1014300089839A83AB83BC8386E080937E0D00E032
:101440000F2EF6E0EF2EFF24F02DEC0EFD1E102FD8
:101450001F5F812F0E948C29D701A00FB11DFC01B5
:1014600080899189969587958C93012F183078F310
:10147000CE0101960E94463FBEC08091750E9091AC
:10148000760E0696AA27BB2789839A83AB83BC83F3
:1014900087E080937E0D00E00F2EF6E0EF2EFF2414
:1014A000F02DEC0EFD1E802F875F0E948C29D70146
:1014B000A00FB11DFC0180899189969587958C9329
:1014C0000F5F083080F3CE0101960E94463F93C023
:1014D0008091750E9091760E0796AA27BB27898377
:1014E0009A83AB83BC8382E08D8389E080937E0DF9
:1014F00000E00F2EF6E0EF2EFF24F02DEC0EFD1E87
:10150000802F8F5E0E948C29D701A00FB11DFC0196
:1015100080899189969587958C930F5F023080F32F
:10152000CE0101960E94463F66C08091750E909153
:10153000760E0996AA27BB2789839A83AB83BC833F
:1015400084E08D838AE080937E0DCE010E960E940A
:1015500072298889282F3327C901880F991F880F7E
:10156000991F880F991F820F931F280F391F832FF0
:1015700099278E832F838989282F332784E690E04B
:10158000289FA001299F500D389F500D1124852FB1
:10159000992788874987CE0101960E94463F2BC034
:1015A0008091750E9091760E0A96AA27BB278983A3
:1015B0009A83AB83BC8386E08D8310927E0DCE012F
:1015C0000E960E9472291E821F82188619868E85A9
:1015D0009F859C01369527953695279536952795B5
:1015E000892F99278695869586958A872B87CE01A0
:1015F00001960E94463F80917C0D90917D0D009751
:1016000009F479C0019790937D0D80937C0D892B0F
:1016100009F071C08091800D9091810D6AE070E0B9
:101620000E945D6270937D0D60937C0D8091820DB0
:101630009091830DAA27BB2789839A83AB83BC83B0
:1016400088E08D838091BE018E838091840D0E94FD
:10165000162A96958795969587958F838091850D07
:101660000E94162A969587959695879588878091EA
:10167000860D0E94162A9695879596958795898757
:101680008091870D0E94162A969587959695879545
:101690008A878091880D0E94162A9695879596953F
:1016A00087958B878091890D0E94162A969587953C
:1016B000969587958C872091BE018FE79DE0FC0170
:1016C000E20FF11D82850E94162A969587959695C0
:1016D00087958D878091BE01982F9F5F9093BE0163
:1016E0008091960D891718F481E08093BE01CE0198
:1016F00001960E94463F8091770D9091780D00975A
:1017000009F405C101979093780D8093770D892B8B
:1017100009F0FDC0CE010E960E9472298091270E1D
:101720009091280E6AE070E00E945D627093780DDF
:101730006093770D8091290E90912A0EAA27BB27DE
:1017400089839A83AB83BC8388E08D83EE240F2E3C
:10175000F0E8FF2EF02D0E2D802F9927FC01EB5D78
:10176000F14F1681133238F4812F0E942C298823DF
:1017700079F0EF280DC01E3238F4812F0E94D20676
:10178000882331F0EF2804C01E3211F4A499EF2809
:10179000F6940F5F083000F3EE82EE240F2EF0E88F
:1017A000FF2EF02D0E2D802F9927FC01EB5DF14FC0
:1017B0001685133238F4812F0E942C29882379F062
:1017C000EF280DC01E3238F4812F0E94D2068823E4
:1017D00031F0EF2804C01E3211F4A499EF28F694DA
:1017E0000F5F083000F3EF82EE240F2EF0E8FF2E9B
:1017F000F02D0E2D802F9927FC01EB5DF14F1689FE
:10180000133238F4812F0E942C29882379F0EF2895
:101810000DC01E3238F4812F0E94D206882331F089
:10182000EF2804C01E3211F4A499EF28F6940F5F3C
:10183000083000F3E886EE240F2EF0E8FF2EF02D9E
:101840000E2D802F9927FC01EB5DF14F168D133281
:1018500038F4812F0E942C29882379F0EF280DC0BD
:101860001E3238F4812F0E94D206882331F0EF28EF
:1018700004C01E3211F4A499EF28F6940F5F0830CB
:1018800000F3E986EE2410914B0E133250F4812FB1
:101890000E942C29882399F00F2EF0E8EF2EF02DCE
:1018A0000EC01E3240F4812F0E94D206882339F0E8
:1018B00050E8E52A04C01E3211F4A499EF281091D3
:1018C0004C0E133240F4812F0E942C29882389F07A
:1018D00080E4E82A0EC01E3240F4812F0E94D20616
:1018E000882339F0E0E4EE2A04C01E3211F4A499F2
:1018F000EF28EA868E859F856AE070E00E945D622F
:101900006B871C861D86CE0101960E94463F809102
:101910007A0D90917B0D009709F4FCC0019790938C
:101920007B0D80937A0D892B09F0F4C08091DF0D37
:101930009091E00D6AE070E00E945D6270937B0D13
:1019400060937A0D8091E10D9091E20DAA27BB275B
:1019500089839A83AB83BC8388E08D83EE240F2E2A
:10196000F0E8FF2EF02D0E2D802F9927FC01E35279
:10197000F24F1681133238F4812F0E9452298823A6
:1019800079F0EF280DC01E3238F4812F0E94D20664
:10199000882331F0EF2804C01E3211F4A499EF28F7
:1019A000F6940F5F083000F3EE82EE240F2EF0E87D
:1019B000FF2EF02D0E2D802F9927FC01E352F24FC0
:1019C0001685133238F4812F0E945229882379F02A
:1019D000EF280DC01E3238F4812F0E94D2068823D2
:1019E00031F0EF2804C01E3211F4A499EF28F694C8
:1019F0000F5F083000F3EF82EE240F2EF0E8FF2E89
:101A0000F02D0E2D802F9927FC01E352F24F1689FD
:101A1000133238F4812F0E945229882379F0EF285D
:101A20000DC01E3238F4812F0E94D206882331F077
:101A3000EF2804C01E3211F4A499EF28F6940F5F2A
:101A4000083000F3E886EE240F2EF0E8FF2EF02D8C
:101A50000E2D802F9927FC01E352F24F168D133281
:101A600038F4812F0E945229882379F0EF280DC085
:101A70001E3238F4812F0E94D206882331F0EF28DD
:101A800004C01E3211F4A499EF28F6940F5F0830B9
:101A900000F3E986EE241091030E133250F4812FE7
:101AA0000E945229882399F00F2EF0E8EF2EF02D96
:101AB0000EC01E3240F4812F0E94D206882339F0D6
:101AC000F0E8EF2A04C01E3211F4A499EF28109117
:101AD000040E133240F4812F0E945229882389F08A
:101AE00020E4E22A0EC01E3240F4812F0E94D2066A
:101AF000882339F040E4E42A04C01E3211F4A4998A
:101B0000EF28EA8688898B871C861D86CE01019680
:101B10000E94463F8091230E9091240E009709F475
:101B20005CC101979093240E8093230E892B09F0BA
:101B300054C18091990D90919A0D6AE070E00E94D5
:101B40005D627093240E6093230E80919B0D9091A3
:101B50009C0DAA27BB2789839A83AB83BC8388E02B
:101B60008D83EE240F2EF0E8FF2EF02D0E2D802F0A
:101B70009927FC01E956F24F1681133238F4812F70
:101B80000E942C29882379F0EF280DC01E3238F4EA
:101B9000812F0E94D206882331F0EF2804C01E3224
:101BA00011F4A499EF28F6940F5F083000F3EE8249
:101BB000EE240F2EF0E8FF2EF02D0E2D802F99270A
:101BC000FC01E956F24F1685133238F4812F0E943A
:101BD0002C29882379F0EF280DC01E3238F4812F8C
:101BE0000E94D206882331F0EF2804C01E3211F47F
:101BF000A499EF28F6940F5F083000F3EF82EE24EB
:101C00000F2EF0E8FF2EF02D0E2D802F9927FC01CE
:101C1000E956F24F1689133238F4812F0E942C298D
:101C2000882379F0EF280DC01E3238F4812F0E94EE
:101C3000D206882331F0EF2804C01E3211F4A49993
:101C4000EF28F6940F5F083000F3E886EE240F2E9D
:101C5000F0E8FF2EF02D0E2D802F9927FC01E9567C
:101C6000F24F168D133238F4812F0E942C298823CD
:101C700079F0EF280DC01E3238F4812F0E94D20671
:101C8000882331F0EF2804C01E3211F4A499EF2804
:101C9000F6940F5F083000F3E986EE240F2EF0E88B
:101CA000FF2EF02D0E2D802F9927FC01E956F24FC3
:101CB00016A1133238F4812F0E945229882379F01B
:101CC000EF280DC01E3238F4812F0E94D2068823DF
:101CD00031F0EF2804C01E3211F4A499EF28F694D5
:101CE0000F5F083000F3EA86EE240F2EF0E8FF2E97
:101CF000F02D0E2D802F9927FC01E956F24F16A5E5
:101D0000133238F4812F0E945229882379F0EF286A
:101D10000DC01E3238F4812F0E94D206882331F084
:101D2000EF2804C01E3211F4A499EF28F6940F5F37
:101D3000083000F3EB86EE240F2EF0E8FF2EF02D96
:101D40000E2D802F9927FC01E956F24F16A9133268
:101D500038F4812F0E945229882379F0EF280DC092
:101D60001E3238F4812F0E94D206882331F0EF28EA
:101D700004C01E3211F4A499EF28F6940F5F0830C6
:101D800000F3EC86EE240F2EF0E8FF2EF02D0E2D42
:101D9000802F9927FC01EB52F24F1081133238F457
:101DA000812F0E945229882379F0EF280DC01E321E
:101DB00038F4812F0E94D206882331F0EF2804C026
:101DC0001E3211F4A499EF28F6940F5F083000F347
:101DD000ED86CE0101960E94463F65960FB6F894B7
:101DE000DEBF0FBECDBFDF91CF911F910F91FF904E
:101DF000EF90089580916B0E90916C0E885E9340E9
:101E000031F084EF91E090936C0E80936B0E8FE035
:101E100090E090936E0E80936D0E89E999E0909317
:101E2000700E80936F0E1092710E1092720E1092BF
:101E3000730E1092740E1092760E1092750EEBE6E1
:101E4000FEE0A0E7B0E08CE090E021E08030920777
:101E500019F40E9411630895182E0E9411630895C9
:101E6000BF92CF92DF92EF92FF920F931F93CF9387
:101E7000DF93CDB7DEB7AE970FB6F894DEBF0FBED7
:101E8000CDBFBB24BE016F5F7F4F8B2D0E94E93019
:101E90008B2D99279C0122953295307F3227207F08
:101EA0003227B90162537E4F9981492F4170DB017E
:101EB0008C91887F9670842B892B8C930F2EFFEB4F
:101EC000CF2EF1E0DF2EF02DC20ED31E8A819B8132
:101ED000F601918380838C819D81938382834E81DF
:101EE0005F81558344838885998597838683D9014B
:101EF000A953BE4F2A858B85982F9295907F822F6C
:101F00008F70892B8C938C8581878D8582878E85B8
:101F100083878F8584878F8D8170982F990F990F74
:101F2000990FFB018081877F892B808388A1F6012F
:101F3000858789A186878AA18170982F9295907F45
:101F4000FB0180818F7E892B80838C918F70833001
:101F500090F5CA01AA2797FDA095BA2FBC01CD0123
:101F60000E94755FDC01CB0128A539A54AA55BA5B8
:101F7000BC01CD010E948F5E7B018C018CA599274D
:101F800087FD9095A92FB92FBC01CD010E94755FE7
:101F9000DC01CB019C01AD01C801B7010E945A5E72
:101FA000DC01CB01BC01CD010E94DB5CDC01CB017B
:101FB000F601958384838B2D99279C012295329578
:101FC000307F3227207F3227F901E953FE4F80818D
:101FD00082958F708330D8F50F2EFFEBCF2EF1E076
:101FE000DF2EF02DC20ED31E88859985AA2797FD76
:101FF000A095BA2FBC01CD010E94755FDC01CB0119
:1020000028A539A54AA55BA5BC01CD010E948F5E1C
:102010007B018C018CA5992787FD9095A92FB92F5D
:10202000BC01CD010E94755FDC01CB019C01AD01BB
:10203000C801B7010E945A5EDC01CB01BC01CD0191
:102040000E94DB5CDC01CB01F601978386832B2D9C
:102050003327C90182959295907F9827807F982792
:10206000FC01E253FE4F808186958370813029F414
:10207000F901E154FC4F808306C08B2D9927FC01A8
:10208000E154FC4F10828B2D9927880F991FFC017A
:10209000E251FC4F11821082B394FFE1FB1508F06E
:1020A000F1CEFE01BD96AAEEB8E082E090E021E01C
:1020B0008030920719F40E94006303C0182E0E941A
:1020C00000638DA58093EC038EA58093ED031092A1
:1020D000E0031092DF03AE960FB6F894DEBF0FBE9A
:1020E000CDBFDF91CF911F910F91FF90EF90DF90C7
:1020F000CF90BF9008951F93CF93DF93CDB7DEB7F6
:10210000AE970FB6F894DEBF0FBECDBF10E0A89516
:102110008981887F89831B821A821D821C821F828B
:102120001E82198618861A861B861C8681E08D877A
:102130001E868F871F8E18A219A21AA280E090E037
:10214000A0E8BFE388A799A7AAA7BBA71CA685E01C
:10215000FE01B39611928A95E9F78FE0FE01709621
:10216000DF01282F1D922A95E9F7189FC00111243D
:1021700086559E4FBC01CF010E940062BE016F5F79
:102180007F4F812F0E94B1301F5F103208F4BFCF04
:102190001EA61DA6FE01BD96AAEEB8E082E090E064
:1021A00021E08030920719F40E94116303C0182EB9
:1021B0000E941163AE960FB6F894DEBF0FBECDBF7E
:1021C000DF91CF911F9108958093DF0308950F93BE
:1021D000CF93DF93CDB7DEB721970FB6F894DEBF6C
:1021E0000FBECDBF89838150803270F000E021E0C6
:1021F000AE014F5F5F4F69E071E082E091E00E94C5
:10220000B42C80E090E007C089819927FC01E2545A
:10221000FC4F8081992721960FB6F894DEBF0FBE40
:10222000CDBFDF91CF910F9108958091EC0388236A
:1022300081F08091ED030E942541882351F4482FBD
:102240008FEB93E0FC01E40FF11D10824F5F4032F1
:10225000C8F340E06EEE73E0AFEBB3E051E0242F43
:102260003327C901820F931FFC01E60FF71F8081FE
:102270009181009709F1019791838083892BE1F483
:10228000C90182959295907F9827807F9827FC01BD
:10229000E253FE4F808186958370992781309105A6
:1022A00039F0029749F0F901EA0FFB1F108204C0D0
:1022B000FD01E40FF11D50834F5F403280F208951D
:1022C0008091DF03882399F08091E003882379F0DF
:1022D00080EE93E0AC014C5F5F4F6091E30380912F
:1022E000E1039091E2030E949E4E1092E003089554
:1022F0008F929F92AF92BF92CF92DF92EF92FF9216
:102300000F931F93CF93DF938C01EE24FF24992426
:102310008091EC03882339F08091ED030E942541E0
:10232000882309F432C280916F0E9091700E9C0147
:1023300044275527F80180819181A281B3818217BA
:102340009307A407B50799F48091710EE80FF11D6A
:1023500085819091720E8923891749F40E94375024
:102360000E94EA1F1092880E82E28093120160E0C0
:102370007091DF030F2EFFEBAF2EF3E0BF2EF02D99
:1023800088248394C0906D0ED0906E0E862F99276E
:1023900082959295907F9827807F9827EC01C15471
:1023A000DE4F88819981AA2797FDA095BA2FF80161
:1023B000208131814281538182179307A407B50799
:1023C00059F08A819B81AA2797FDA095BA2F821781
:1023D0009307A407B507C1F4462F5527CA01840FF8
:1023E000951FFC01E251FC4FD182C082872F7330D0
:1023F00048F099279C012F733070CA010396281763
:10240000390711F4992493948F8583FF09C08D8532
:10241000F801E80FF11D9E858581981709F062C1CA
:10242000288139812115310509F45CC1442737FD24
:102430004095542FF80180819181A281B3812817A2
:1024400039074A075B0709F09DC091E08985882319
:1024500079F0E80FF11D8481E82EFF24FE2CEE2494
:102460008A85F801E80FF11D8481E80EF11C14C083
:102470008A85882381F0F801E80FF11D8481E82E18
:10248000FF248F8584FF08C0EE2034F420E03FEF66
:10249000E22AF32A01C090E0992309F473C08885E9
:1024A0008F70992782309105B9F1833091052CF412
:1024B000009779F00197C1F065C08430910509F467
:1024C0004DC0843091050CF43EC0059709F451C00D
:1024D00059C08C819D818E159F0509F053C0F5016F
:1024E000E60FF11D80824EC08F8584FF0BC08C816A
:1024F0009D818E159F050CF045C0F501E60FF11D7D
:10250000808240C08C819D818E159F05D8F5F50194
:10251000E60FF11D808236C08F8584FF0AC08C8152
:102520009D81E816F90674F5F501E60FF11D80822C
:1025300029C08C819D81E816F90620F5F501E60F8A
:10254000F11D80821FC08C819D818E219F21892B4E
:10255000C9F0F501E60FF11D808214C08C819D81C8
:102560008E219F21892B71F4F501E60FF11D8082E8
:1025700009C08C819D818E159F0521F0F501E60F24
:10258000F11D80828A819B819C01442737FD409503
:10259000542FF80180819181A281B38128173907D6
:1025A0004A075B0709F09EC091E08B85882379F08C
:1025B000E80FF11D8481E82EFF24FE2CEE248C858B
:1025C000F801E80FF11D8481E80EF11C14C08C8520
:1025D000882381F0F801E80FF11D8481E82EFF24A3
:1025E0008F8584FF08C0EE2034F420E03FEFE22A1C
:1025F000F32A01C090E0992309F474C0888582957C
:102600008F70992782309105B9F1833091052CF4B0
:10261000009779F00197C1F065C08430910509F405
:102620004DC0843091050CF43EC0059709F451C0AB
:1026300059C08E819F818E159F0509F053C0F50109
:10264000E60FF11D10824EC08F8584FF0BC08E8176
:102650009F818E159F050CF045C0F501E60FF11D19
:10266000108240C08E819F818E159F05D8F5F5019F
:10267000E60FF11D108236C08F8584FF0AC08E815F
:102680009F81E816F90674F5F501E60FF11D108239
:1026900029C08E819F81E816F90620F5F501E60F25
:1026A000F11D10821FC08E819F818E219F21892B59
:1026B000C9F0F501E60FF11D108214C08E819F81D3
:1026C0008E219F21892B71F4F501E60FF11D1082F7
:1026D00009C08E819F818E159F0521F0F501E60FBF
:1026E000F11D10826F5F603208F450CE8091DF03DD
:1026F000882309F44AC0992019F4823009F045C0B2
:102700008091E003823009F440C08091E103909110
:10271000E2039C0144275527F80180819181A28121
:10272000B381281739074A075B0799F49091E303AF
:102730008481981771F4892F992798012B5F3F4F57
:10274000AC01B90180EE93E004960E940762892BE8
:10275000C9F082E08093E003F80124812093E30331
:10276000808191819093E2038093E103822F9927E6
:1027700098012B5F3F4FAC01B90184EE93E00E94BA
:10278000146203C081E08093E003DF91CF911F9139
:102790000F91FF90EF90DF90CF90BF90AF909F9000
:1027A0008F9008950E948D058091D800826080935B
:1027B000D8000895CF93DF93EC018981833089F4A9
:1027C0008985882309F403C188818295807F80935D
:1027D000ED008091EF008F738093EF0018821986CF
:1027E000F6C00E94B105982F81E089879F3F09F4C8
:1027F000EBC09883892F8295807F8093ED001092A3
:10280000EE001092EF001092F7001092F600109276
:10281000F5001092F4001092F00089819927813020
:10282000910509F46BC0823091051CF4892B29F0C5
:10283000C9C0029709F4BBC0C5C08A8581FF30C0FA
:102840008D81982F990F990F990F8C81829586957C
:102850008770890F8093F3008C81982F990F990FBF
:10286000990F8B81829586958770890F8093F200EE
:102870008B81982F990F990F990F8A818295869550
:102880008770890F8093F1008A81880F880F880FE5
:102890008093F0008091EF0080618093EF0012C080
:1028A0008B81982F9295990F907E8A818695869537
:1028B0008695890F8093F3008A818295880F807EA8
:1028C0008093F20020E08E81181660F48F81988545
:1028D000FC01E20FF11D80818093FA002F5F8E8151
:1028E0002817A0F39091EF008E81892B8093EF0041
:1028F0008091EF0080648093EF0069C08A8581FF3A
:1029000035C08D81982F990F990F990F8C818295E1
:1029100086958770890F8093F3008C81982F990F8B
:10292000990F990F8B81829586958770890F809377
:10293000F2008B81982F990F990F990F8A818295B8
:1029400086958770890F8093F1008A81880F880FA0
:10295000880F8093F0008091EF0080618093EF00FA
:102960008091F00084608093F00015C08B81982FD7
:102970009295990F907E8A81869586958695890F86
:102980008093F3008A818295880F807E8093F20085
:1029900084E08093F0009091EF008E81892B8093EA
:1029A000EF008091EF0080648093EF0010C0809171
:1029B000EF008F738093EF008091EF008068809329
:1029C000EF0005C0198603C08FEF90E002C080E0E1
:1029D00090E0DF91CF910895CF93DF93EC0189854B
:1029E000882319F482E090E082C088818295807FFC
:1029F0008093ED000E94CB05813009F06CC01986F0
:102A00008091EF008F708E838F8198850E94E305FF
:102A10008091F00099278470907095958795959591
:102A20008795982F91708A85282F2E7F292B2A87AA
:102A30008091EF0084FF31C0822F82608A8780916D
:102A4000F3008695869586958D838091F200982F68
:102A50009695969596958091F3008295880F807E45
:102A6000890F8C838091F100982F96959695969575
:102A70008091F2008295880F807E890F8B838091F0
:102A8000F000982F9695969596958091F1008295F5
:102A9000880F807E890F8A8316C08A858D7F8A87FA
:102AA0008091F3008295869587708B838091F200E8
:102AB000982F9295969597708091F300880F880FC4
:102AC000880F890F8A838091EF008F738093EF00C6
:102AD00080E090E00CC0882349F489878091EF0062
:102AE0008F738093EF0080E090E001C09927DF9121
:102AF000CF910895982F8F3F19F481E090E00895C9
:102B0000805C843128F4892F0E94254199270895FB
:102B1000892F8150803228F4892F0E94E71099274D
:102B20000895892F8152843128F4892F0E947F547F
:102B30009927089580E090E008958091790E0E9491
:102B40007A15882321F085E08093E70941C08091C0
:102B50007E0E0E947A15882341F080917F0E80932B
:102B6000E90983E08093E70933C08091780E0E94E1
:102B70007A15882321F084E08093E70929C08091A9
:102B80007A0E0E947A15882341F08091E7098730F8
:102B900021F086E08093E7091BC08091E70985302A
:102BA00021F482E08093E70913C08091E709833024
:102BB00041F48091E909882321F481E08093E709B9
:102BC00007C08091E709843019F481E08093E70918
:102BD0008091E7098150823058F480917B0E0E94E9
:102BE0007A1590917C0E981719F41092E70913C08A
:102BF0008091E709863079F480917B0E0E947A15E6
:102C000090917C0E981739F487E08093E7098091C2
:102C10007D0E8093E80982E699E00E940C2B0E94C9
:102C2000C41708951F93CF93DF9310E0812F992746
:102C3000EC01C80FD91FFE01E058F14F80818823B5
:102C400009F4B4C00E947A15882309F4AFC0FE01CC
:102C5000EF57F14F808183FDB3C088608083877018
:102C600099278230910539F1833091051CF4019741
:102C700029F0A6C0039709F452C0A2C0812F99275A
:102C8000880F991FFC01EF57F14F9081892F829592
:102C90008F70877021F0892F8F78808391C0812F6A
:102CA0009927880F991FFC01EF57F14F80818F788A
:102CB0008061808385C0812F9927880F991FFC012F
:102CC000EF57F14F808182958F7087709927009719
:102CD00019F0019769F018C0812F9927880F991F63
:102CE000FC01EF57F14F80818F788061808368C04D
:102CF000812F9927880F991FFC01EF57F14F808191
:102D00008F78806280835CC0812F9927880F991FFC
:102D1000FC01EF57F14F80818F78808351C0812F64
:102D20009927880F991FFC01EF57F14F80818295F9
:102D30008F708770992781309105A9F082309105B5
:102D40001CF4892B21F027C00297C9F024C0812FE1
:102D50009927880F991FFC01EF57F14F80818F78D9
:102D6000806180832DC0812F9927880F991FFC01D6
:102D7000EF57F14F80818F788062808321C0812F4F
:102D80009927880F991FFC01EF57F14F80818F78A9
:102D90008063808315C0812F9927880F991FFC01BC
:102DA000EF57F14F80818F7880830AC0812F992758
:102DB000880F991FFC01EF57F14F8081877F808337
:102DC0001F5F143008F432CF0E94BE200E94531FB0
:102DD0000E94392210E085E2189FC0011124EC0105
:102DE000CB5CDB4F8C899D89009719F001979D8BF7
:102DF0008C8B8D859E85009761F001979E878D87CE
:102E000099859F3F31F085E0989FC00111249B87F1
:102E10008A872A853B852115310561F089858F3F99
:102E200049F0C90101979B878A87892B19F48F85FF
:102E300080628F878A8D9B8D009779F001979B8F99
:102E40008A8F892B51F48F8586FD04C0812F8F5F77
:102E50000E94922F8F8580648F878F81882311F045
:102E600081508F831F5F123208F4B5CFDF91CF916D
:102E70001F9108958091E7098730A1F48091E809B6
:102E8000882321F081508093E8090CC080917A0E4C
:102E90000E947A15882321F086E08093E70902C01A
:102EA0001092E7098091E909882319F081508093F5
:102EB000E909A49B23C02091E4092F3710F4220FC5
:102EC00001C02FEF8091730E8A30D0F09091770E71
:102ED000981710F0921730F48091770E8F5F8093DF
:102EE000770E0EC08091880E882351F48F5F8093F7
:102EF000880E0E9437500E94EA1F02C01092770E7F
:102F000090915909809169099817E0F420E049E609
:102F100059E065E270E0FA01E20FF11D8281823230
:102F200068F49927869FF001879FF00D969FF00D1A
:102F30001124E75CFB4F8081816080832F5F2C3000
:102F400050F308959091590980916A098917D8F42E
:102F500020E049E659E065E270E0FA01E20FF11D78
:102F60008281823268F49927869FF001879FF00D55
:102F7000969FF00D1124E75CFB4F80818E7F80834C
:102F80002F5F2C3050F30895CF92DF92EF92FF9293
:102F90000F931F93CF93DF9380912F04882309F021
:102FA00004C1F82E0F2EFAE0EF2EF02D8EE0F89EE1
:102FB000C0011124EC01C256D64F00E08A818F3F38
:102FC00011F401E01DC09A81892F805C843128F4BE
:102FD000892F0E942541082F13C09A81892F815083
:102FE000803228F4892F0E94E710082F09C09A81A7
:102FF000892F8152843120F4892F0E947F54082F19
:103000008981992781309105C9F1823091051CF49D
:10301000892B29F0C5C0029709F4BFC0C1C0013097
:1030200009F0BEC08F818E9DC00111249C838B83CB
:1030300089858E9DC00111249E838D838881846043
:10304000888310E025E230E0FE01E10FF11D82856A
:103050008F3F71F09927829FA001839F500D929F0F
:10306000500D1124FA01E75CFB4F8081846080835E
:103070001F5F143048F381E0898392C08B819C816B
:10308000009709F48DC001979C838B83892B81F570
:10309000288122FF17C08F818E9DC00111249C833F
:1030A0008B83822F8B7F888310E0FE01E10FF11D5F
:1030B00082858F3F19F060E00E94DE181F5F143098
:1030C000A0F316C088858E9DC00111249C838B833C
:1030D00088818460888310E0FE01E10FF11D828504
:1030E0008F3F19F061E00E94DE181F5F1430A0F3DB
:1030F0008881282F227081FD28C08D819E810097B4
:1031000009F44EC001979E838D83892B09F048C036
:1031100082E08983122F25E230E0FE01E10FF11DEC
:1031200082858F3F71F09927829FA001839F500D68
:10313000929F500D1124FA01E75CFB4F80818B7F39
:1031400080831F5F143048F32BC0002349F5102FF4
:103150000F2EF5E2CF2EDD24F02DFE01E10FF11D43
:1031600022852F3F99F0822F99278C9DA0018D9D5C
:10317000500D9C9D500D1124FA01E75CFB4F80819E
:103180008B7F808361E0822F0E94DE181C821B826D
:103190001F5F143010F3198203C0002309F4098360
:1031A000F39454E05F1508F001CFDF91CF911F91A8
:1031B0000F91FF90EF90DF90CF900895DF92EF9204
:1031C000FF920F931F93CF93DF93CDB7DEB7219775
:1031D0000FB6F894DEBF0FBECDBF8983162FDD2456
:1031E000833260F00D2D21E0AE014F5F5F4F61E74C
:1031F00072E083E191E00E94B42C4EC0998185E297
:10320000989F7001112485E394E0E80EF91EF70100
:10321000858D9927807F9070803A910529F40F2E33
:10322000F1E4DF2EF02D18C0F701858D9927807FFE
:103230009070803B910529F40F2EF2E4DF2EF02DE3
:103240000BC000E021E0AE014F5F5F4F6DE772E021
:1032500083E191E00E94B42C112379F483E0F7011B
:10326000878380EF818387858F7B8787858D41A1C9
:103270006D2D8F700E949A390FC0113069F4F701DB
:1032800017828FE08183878586798787858D41A125
:103290006D2D8F700E94E53921960FB6F894DEBF30
:1032A0000FBECDBFDF91CF911F910F91FF90EF9097
:1032B000DF90089520E047E759E065E270E0817013
:1032C000382F330FFA01E20FF11D8181823270F441
:1032D0009927869FF001879FF00D969FF00D11248E
:1032E000E75CFB4F80818D7F832B80832F5F2E30A7
:1032F00048F3089520E047E759E065E270E0817007
:10330000382F330FFA01E20FF11D8189823270F4F8
:103310009927869FF001879FF00D969FF00D11244D
:10332000E75CFB4F80818D7F832B80832F5F2E3066
:1033300048F308958091310490913204089580916A
:10334000300499270895EF92FF921F93CF93DF9354
:103350007A018093690960936A0910E0C12FDD2723
:10336000F701EC0FFD1F80810E949927823220F423
:10337000FE01E759F64F82831F5F1C3078F3DF911F
:10338000CF911F91FF90EF9008957F928F929F921F
:10339000AF92BF92CF92DF92EF92FF920F931F9363
:1033A000CF93C0E00E949A290E94892A0E94B42AE1
:1033B00082E699E00E94012B10925709109256095B
:1033C000C0935809C0935A09C0935B09C0935C0924
:1033D000C0935D0982E1EFE1F9E011928A95E9F786
:1033E00041E359E028EB31E08C2F9927880F991F92
:1033F000FC01E40FF51F31832083CF5FC231A0F3BE
:10340000C0E04EE959E02EE030E08C2F9927829FF2
:10341000B001839F700D929F700D1124FB01E40F8A
:10342000F51F11821482138216821582FB01E25667
:10343000F64F808184608083CF5FC53030F30E9477
:103440004133803221F487E68093110103C08EE678
:1034500080931101A5E3B4E041E04093350428ECEA
:1034600030E0309348042093470452EA50935204CA
:1034700062EB60935304109256049FEF90935404B0
:103480005093550483E0809357048D010B5D1F4FCB
:1034900040935A04FD0130AF27ABF801558F668F7A
:1034A00041A3978F0F2EF7EAEF2EF02DE0A20F2EFB
:1034B000FFE0BF2EF02DB2A2FD01E65BFF4F40936F
:1034C0007F04338B228B0F2EF3EADF2EF02DD58E67
:1034D00083EB868F41A3978F90A389E082A3FD01A0
:1034E000E159FF4F4093A404338B228BE58E0F2EBE
:1034F000F7EBCF2EF02DC68E41A3978F90A38BE0D4
:1035000082A3FD01EC56FF4F4093C904338B228BFD
:1035100011EA158F0F2EF1EBFF2EF02DF68E41A341
:10352000978F90A38EE082A3FD01E754FF4F409355
:10353000EE04338B228B55EA558F05EB068F41A3A2
:10354000978F90A38DE082A3C6E0FD01E252FF4F6A
:1035500040931305338B228B60EA658F70EB768F77
:1035600011A2978F50A3C2A3FD01ED5FFE4F4093C0
:103570003805338B228B558F068F11A2978F90A31E
:1035800084E082A3FD01E85DFE4F40935D05338B2F
:10359000228B658F768F41A3978F60A38AE082A3E9
:1035A000FD01E35BFE4F40938205338B228B758FC9
:1035B00054EB568F75E071A3978F90A382E182A39D
:1035C000FD01EE58FE4F4093A705338B228B64EA32
:1035D000658F568F41A3978FD0A288E082A3FD010B
:1035E000E956FE4F4093CC05338B228B56EA558F1C
:1035F00086EB868F11A2978F60A342A3CCE0FD01DA
:10360000E454FE4F4093F105338B228B558F868F08
:1036100041A3978F10A3C2A3FD01EF51FE4F40932A
:103620001606338B228BE58EC68E11A2978F90A340
:1036300082E082A3FD01EA5FFD4F40933B06338B9E
:10364000228B158FF68E11A2978F90A387E082A30D
:10365000FD01E55DFD4F40936006338B228BF58EB7
:10366000068F71A3978F2B2D3327AD0185E290E054
:10367000289FB001299F700D389F700D1124FB0108
:10368000EA0FFB1F9FEF90A381E182A3FD01E05BA6
:10369000FD4F61E06093850628EC30E0338B228B90
:1036A000B4EAB58F0F2EF4EBFF2EF02DF68E11A29B
:1036B000978F0F2EF6EAEF2EF02DE0A285E082A381
:1036C000FA01EB58FD4F6093AA06338B228B8D2CA9
:1036D000D58E03EB068F11A2978F90A312A2FA0149
:1036E000E656FD4F70E47093CF062FEF3FEF338B1C
:1036F000228B0F2EF7EADF2EF02DD58EF68E63E0AB
:1037000061A3E78E90A392A3FA01E154FD4F709359
:10371000F406338B228BE58E15EB168F61A3E78EB3
:1037200090A392A3FA01EC51FD4F70931907338BCC
:10373000228BA5EAA58F0F2EF6EB7F2EF02D768E2D
:1037400061A3D78E90A392A3FA01E75FFC4F709319
:103750003E07338B228BB58FC68E61A3D78E90A385
:1037600092A3FA01E25DFC4F70936307338B228BC7
:1037700080EA858F068F61A3A78F90A392A3FA0199
:10378000ED5AFC4F70938807338B228B0F2EF1EA92
:10379000BF2EF02DB58E0F2EF2EBAF2EF02DA68E94
:1037A00061A3A78F90A392A3FA01E858FC4F7093EE
:1037B000AD07338B228B0F2EF2EA9F2EF02D958EC4
:1037C000A1EBA68F61A3B78F90A392A3FA01E35652
:1037D000FC4F7093D207338B228B858E0F2EF0EB2C
:1037E000CF2EF02DC68E61A3B78F90A392A3FA01BE
:1037F000EE53FC4F7093F707338B228B858F068F28
:1038000082E081A3178F90A392A3FA01E951FC4FA4
:1038100070931C08338B228BB58EA68E81A3178FD5
:1038200090A392A3FA01E45FFB4F70934108338B9E
:10383000228B958EA68F81A3F78E90A392A3FA0177
:10384000EF5CFB4F70936608338B228B858EC68EA0
:1038500081A3F78E90A392A3FA01EA5AFB4F7093CB
:103860008B08338B228BD58EF68E81A3778E90A317
:1038700092A3FA01E558FB4F7093B008338B228B6B
:10388000E58EFA01E558FB4F168F9A01FA01E558CB
:10389000FB4F52E051A3778E4FEF40A342A3F901B3
:1038A000E056FB4FA72F7093D5086FEF7FEF738B18
:1038B000628B85EA858F768E51A397EB978F40A315
:1038C00042A3F901EB53FB4FA093FA08738B628B71
:1038D000B58F968F51A3978F40A342A3C0E0B90143
:1038E00045E250E02FE001E21EE130E18C2F992704
:1038F000849FF001859FF00D949FF00D1124CF015E
:10390000E60FF71F158A148ADC01A75CBB4F8C9168
:103910008C7D8C931786168A218314A213A2168697
:10392000158614861386128611868C918B7F8C9354
:10393000178A17820087168335832283118E108E93
:10394000138E128E148ECF5FC23280F2CF911F91F0
:103950000F91FF90EF90DF90CF90BF90AF909F902E
:103960008F907F900895EFE1F9E082E1DF011D92F1
:103970008A95E9F7CF010E94733220E061E379E094
:1039800048EB51E0822F9927880F991FFC01E60F21
:10399000F71F518340832F5F2231A0F381E399E029
:1039A0000E9493320895AF92BF92CF92DF92EF922E
:1039B000FF920F931F93CF93DF93CDB7DEB7C35C16
:1039C000D0400FB6F894DEBF0FBECDBF10E00F2E73
:1039D000F5E6EF2EFF24F02DEC0EFD1E212F3327F0
:1039E00085E290E0289FA001299F500D389F500D3F
:1039F00011249A012B5C3B4FF90182899389892F0D
:103A00009927D7018C938289F7018183F9018681F7
:103A1000F7018283158214821682F9018581F701EC
:103A20008383F9018085F70187838FE0189FC001A8
:103A3000112486589B4FBC01C70108960E94006262
:103A4000F701178A108E1F5F612FC7010E94913105
:103A5000A895123218F28E0102581F4F84E6D80141
:103A60008C9388E7F80181834CE050E06FEF70E0C1
:103A7000C80102960E942162C8010E94D12F8E01C6
:103A800004571F4FF80181EC81934EE050E06FEF37
:103A900070E0CF010E942162F80117868AE0808BD6
:103AA0004EE050E06FEF70E0C80141960E94216245
:103AB000C8010E94FF2FA89510E00F2EF4E1DF2E21
:103AC000F02D7E010894E11CF11C0FE0D701ED2DD3
:103AD0001D92EA95E9F7109FC00111248B529C4F6B
:103AE000BC01C7010E940062188A1F5FB701812FC5
:103AF0000E9428321B3050F3A89510E00F2EF5EBF2
:103B0000AF2EBB24F02DAC0EBD1E0F2EFFE0CF2E2E
:103B1000F02D0F2EFBEAEF2EFF24F02DEC0EFD1EF4
:103B2000DD24D3940FEFD501EC2D1D92EA95E9F732
:103B30001C9DC001112486579C4FBC01C7010A96E9
:103B40000E940062D7011C92F70111821282D38277
:103B5000D4828AE085838081F701E80FF11D068316
:103B60008F5F8430C8F3BE0165557F4F812F0E945F
:103B70003F301F5F1530B8F2E6E9F9E018E0DF01E9
:103B8000212F1D922A95E9F7CF010E941F300E9434
:103B90007C2AA895E8E7FEE0DF011D921A95E9F777
:103BA00081E080937C0E8EE180937D0E82E3809392
:103BB0007F0EAEE6BFE088E090E021E08030920723
:103BC00019F40E94116303C0182E0E9411639E0114
:103BD0002B5E3F4F8CE4D9011D928A95E9F78CE06A
:103BE000A1E2B1E0FE017796482F0D9001924A952F
:103BF000E1F7ADE2B1E0FE01BA96582F0D900192C7
:103C00005A95E1F7A9E3B1E0FE01FD96982F0D90DA
:103C100001929A95E1F7A5E4B1E0FE01E05BFF4F68
:103C20000D9001928A95E1F7F901AEE8BFE08CE4CE
:103C300090E021E08030920719F40E94116303C0E4
:103C4000182E0E94116388E0E0E8FEE011928A9548
:103C5000E9F7CD53DF4F0FB6F894DEBF0FBECDBFEF
:103C6000DF91CF911F910F91FF90EF90DF90CF9058
:103C7000BF90AF900895CF92DF92EF92FF920F9393
:103C80001F93CF93DF93CDB7DEB7E4970FB6F894C9
:103C9000DEBF0FBECDBF00E0102F1F5F612FCE0132
:103CA00001960E94D631202F332785E290E0289F8D
:103CB000A001299F500D389F500D1124FA01EB5C93
:103CC000FB4F89819927982F88272A81820F911D80
:103CD000938B828B8B818683888580878C8185837B
:103CE000888D8487898D81878D819E81918F808F3A
:103CF0008F81848F012F123278F289E699E00E9439
:103D0000EF2F87E799E00E940F308FE199E00E9442
:103D1000833281E399E00E94A33286E999E00E9410
:103D20002F300E947C2A00E0BE01665E7F4F802F0C
:103D30000E947830202F33278EE090E0289FF001FA
:103D4000299FF00D389FF00D11249F01E256F64F88
:103D50008A8D582F51708081482F4C7F8B8D8170B8
:103D6000982F990F842F852B892B8083F901E25698
:103D7000F64F8C8D82838D8D87838E8D80878F8D7E
:103D80008187F901E855F64F88A199A1AAA1BBA1A5
:103D900080839183A283B3830F5F053028F2E8E725
:103DA000FEE0AEE6BFE088E090E021E080309207E0
:103DB00019F40E94006303C0182E0E94006300E003
:103DC00073E142E050E0642F0F2EF0E8CF2EFEE0CA
:103DD000DF2EF02D0F2EF3E3EF2EFF24F02DEC0E4F
:103DE000FD1EFE01F396079FC0011124DC01A257BE
:103DF000B04F4115510551F081E04030580719F49A
:103E00000E94006303C0162E0E940063802F992732
:103E10009C01280F391FF901EC0DFD1D8BA9808332
:103E2000D901AF57B14FF7018181982F97708C91CD
:103E30008078892B8C930F5F043098F2E4960FB64C
:103E4000F894DEBF0FBECDBFDF91CF911F910F91D0
:103E5000FF90EF90DF90CF900895CF93DF93EC0128
:103E6000862F0E9499278332D8F4282F332785E2A2
:103E700090E0289FA001299F500D389F500D1124DC
:103E8000FA01EB5CFB4F8F89848788819927982FF3
:103E900088272981820F911D938B828B8A8186834B
:103EA000DF91CF9108951F93CF93C0E01C2F909185
:103EB0007709892F8150803238F4892F0E94E710CA
:103EC0008823B1F011E014C090917709892F8152B5
:103ED000843138F4892F0E947F54882349F011E0FF
:103EE00007C0809177090E942541813009F4182F7D
:103EF00090918609892F8150803220F4892F0E9469
:103F0000E7100EC090918609892F8152843120F4E8
:103F1000892F0E947F5404C0809186090E94254108
:103F20008E3FF1F08130B9F48091E509843020F4BE
:103F30008F5F8093E50909C01092E5098091E60939
:103F4000882319F081508093E6098091E60988233F
:103F500059F4C1E009C0809187098093E60904C043
:103F6000809187098093E609113021F4812F0E9406
:103F70005A190CC0C13021F48C2F0E947A1906C046
:103F800080E00E945A1980E00E947A19CF911F9117
:103F90000895FC018481982F986080EF8283878543
:103FA00086798787168A892F8F7D8483848525E08B
:103FB000829FC001112496878587892B41F48185D2
:103FC0008F3F29F0829FC00111249387828783E06D
:103FD000878308951F93CF93C0E015E2C19FC0016E
:103FE0001124FC01EB5CFB4F8785992783FD02C000
:103FF00080FF03C0CF010E94C91FCF5FC23270F3A0
:10400000CF911F91089599278C33910509F466C0CB
:104010008D339105A4F488339105A1F1893391057D
:104020001CF4C79721F1A7C089339105B1F18A33F8
:10403000910509F43DC0CB9709F445C09CC080347C
:10404000910509F477C08134910544F48E339105CC
:1040500009F45AC0CF970CF062C04BC0813491056F
:1040600009F473C08234910509F47AC084C0809148
:10407000810E8077803119F481E090E0089580E02E
:1040800090E008958091810E8077803219F481E06C
:1040900090E0089580E090E008958091810E80770F
:1040A000803319F481E090E0089580E090E0089575
:1040B0008091830E8077803119F481E090E008953B
:1040C00080E090E008958091830E8077803219F42B
:1040D00081E090E0089580E090E008958091830E63
:1040E0008077803319F481E090E0089580E090E0DB
:1040F00008958091850E8077803119F481E090E0F9
:10410000089580E090E008958091850E8077803258
:1041100019F481E090E0089580E090E008958091A6
:10412000850E8077803319F481E090E0089580E077
:1041300090E008958091870E8077803119F481E0B6
:1041400090E0089580E090E008958091870E807758
:10415000803219F481E090E0089580E090E00895C5
:104160008091870E8077803319F481E090E0089584
:1041700080E090E0089580E090E00895FF920F9332
:104180001F93CF93DF9310E00F2EFFE0FF2EF02D53
:1041900082E00E94CB4185E2189FC0011124EC010E
:1041A000CB5CDB4F8885882361F48981803F09F0EF
:1041B000F4C08C8188608C838F85867B8F87FA82A0
:1041C000ECC02885822F81508032D0F58F859927C9
:1041D00083FD24C080FD22C0822F0E94E710882327
:1041E00041F089818F3009F0D8C0CE010E94C91FEB
:1041F000D4C08981803F09F0D0C089858F3F09F400
:10420000CCC08A859B85892B09F0C7C08C818860CA
:104210008C838F85867B8F87FA82BFC088850E94BA
:10422000E710882309F0B9C08981803F09F0B5C043
:104230008C8188608C838F85867B8F87FA82ADC066
:104240002885822F81528431D0F58F85992783FD6F
:1042500024C080FD22C0822F0E947F54882341F019
:1042600089818F3009F099C0CE010E94C91F95C085
:104270008981803F09F091C089858F3F09F48DC005
:104280008A859B85892B09F088C08C8188608C8306
:104290008F85867B8F87FA8280C088850E947F54B5
:1042A000882309F07AC08981803F09F076C08C812B
:1042B00088608C838F85867B8F87FA826EC000E052
:1042C0008885853371F49091E709892F8350823076
:1042D00020F0913011F0963011F491E01DC090E083
:1042E0001BC08885863351F48091E709853011F031
:1042F000823011F491E010C090E00EC09885892FB3
:1043000087538C3028F4892F0E940320982F04C0F3
:1043100088850E942541982F9E3FA9F08885803C82
:1043200021F49130A1F4092F12C08D81813021F444
:10433000913011F4092F0BC08D81803141F4992304
:1043400031F401E004C088858F3F09F401E00023C7
:1043500069F089818F3009F58F85992783FD1DC00C
:1043600080FD1BC0CE010E94C91F17C08981803FFC
:1043700031F08F85992783FD02C080FF0EC08985AB
:104380008F3F59F08A859B85892B39F48C81886011
:104390008C838F85867B8F87FA8289818F3079F431
:1043A0008F85992789709070892B49F4809112012B
:1043B000811729F482E2809312011092880E1F5F08
:1043C000123208F4E5CEDF91CF911F910F91FF904B
:1043D000089560932F04623019F48FEF809355098C
:1043E0000895CF93DF93EC0188818150823218F0D9
:1043F00080E090E03BC088810E949927282F898126
:1044000099278F30910521F0803F9105A1F02CC0B4
:10441000332785E290E0289FA001299F500D389F07
:10442000500D1124FA01EB5CFB4F8FE081838785EF
:10443000867F878719C0332785E290E0289FA001F7
:10444000299F500D389F500D1124FA01EB5CFB4F52
:1044500080EF81838785867F8787168AFA01E75CEC
:10446000FB4F80818F7D808381E090E0DF91CF9151
:1044700008958F929F92AF92BF92CF92DF92EF9268
:10448000FF920F931F93CF93DF93CDB7DEB72197A2
:104490000FB6F894DEBF0FBECDBFBB24B9828B2C04
:1044A000AB2C9B2C1092570910925609B0925A09C6
:1044B000B0925C09B0925B090E9422058093590971
:1044C00080912F04882309F07DC2B9828B2D82321E
:1044D00008F0FAC482E00E94CB418824998185E2E9
:1044E000989FC00111240F2EF5E3CF2EF4E0DF2EAC
:1044F000F02DC80ED91EF601858D9927807F90700A
:10450000803A910529F40F2EF1E4AF2EF02D18C05A
:10451000F601858D9927807F9070803B910529F465
:104520000F2EF2E4AF2EF02D0BC000E021E0AE0123
:104530004F5F5F4F6EE677E083E191E00E94B42C1D
:10454000F601118A108A248122FDBCC0808199273E
:104550008130910509F45DC08034910509F0BFC038
:10456000818199278F309105B1F1803F910509F044
:10457000B6C0822F837019F4878585FF09C0F601C4
:10458000858D41A16A2D8F700E94E539882410C065
:10459000F60185859685892B59F4878580FD08C0AD
:1045A000858D41A16A2D8F700E949A398824839449
:1045B000F601848183FF93C0877F848382818F305B
:1045C00009F08DC08183858D41A16A2D8F700E9475
:1045D000E539882484C0F601248123FF80C0822F1E
:1045E000877F84838281803F09F079C081838585BC
:1045F0009685892B09F073C0822F837009F06FC0F4
:10460000858D41A16A2D8F700E949A3988248394E8
:1046100066C0F601818199278F309105C1F1803FF5
:10462000910509F05CC08481837019F4878585FF4A
:1046300009C0F601858D41A16A2D8F700E94E53970
:10464000882413C0F60185859685892B71F48785AA
:10465000992780FD0AC083FD08C0858D41A16A2D80
:104660008F700E949A3988248394F601848183FF95
:1046700036C0877F848382818F3089F58183858DE1
:1046800041A16A2D8F700E94E539882428C0F60167
:10469000248123FF24C0822F877F84838281803FEF
:1046A000F1F4818385859685892BC9F4822F8370E7
:1046B000B1F4858D41A16A2D8F700E949A398824AA
:1046C00083940DC0F601818199278F30910531F0D7
:1046D000803F910521F48824839401C08824F60149
:1046E0008181803F09F058C082A18F3F09F454C0F6
:1046F0000E94F1037C0100271127F601F4A2E3A236
:1047000089819927FC01E15EF64F80819927AA27CC
:10471000BB278E159F05A007B10724F0EE24FF24C8
:1047200087010AC089819927FC01E15EF64F8081EB
:10473000E81AF10801091109F3E0EF16F104010587
:104740001105CCF089819927880F991FFC01EF5C36
:10475000F64F808191819C0144275527C801B701FC
:104760000E94326220EE31E040E050E00E94A662FA
:1047700079018A0103C0EE24FF248701F601F18A42
:10478000E08A80915609909157098E0D9F1D909354
:1047900057098093560903C0F601118A108A8820B0
:1047A00039F4F601828D938D892B11F0138E128EC0
:1047B000F60187859927AC014870507083FD70C061
:1047C000208931898289938982179307E0F5828D48
:1047D000938D892B11F0538F428FF601848185FFD1
:1047E00026C084899589892B09F05AC087858860FD
:1047F000878780915A098F5F80935A098081813021
:1048000071F4858D41A16A2D8F700E94E53988244D
:10481000898180931201F60186818093E409898160
:10482000F601608971898F5F0E94272F39C0F601D8
:10483000848180628483968185E0989FC0011124E1
:10484000958B848B2DC0F60184818F7D8483208D90
:10485000318D2115310521F18820A1F080899189C0
:104860008217930778F4828D938D892BC9F48785FD
:1048700086FD16C0948D85E0989FC0011124938F0A
:10488000828F0EC0F601828D938D892B49F020898D
:104890003189808D918D8217930710F4138E128EBB
:1048A000F601868D9927807F9070803A910529F4D2
:1048B0000F2EF1E49F2EF02D18C0F601868D99275A
:1048C000807F9070803B910529F40F2EF2E49F2E9B
:1048D000F02D0BC000E021E0AE014F5F5F4F66E8B6
:1048E00078E083E191E00E94B42CF601868D41A12D
:1048F000692D8F700E94683A282FF6018181803FD0
:1049000009F043C08785992783FD3FC080FD3DC0E6
:1049100090915909809111018917B8F5F1E08F162E
:1049200091F5222381F5F6018781882371F584852D
:10493000882359F587898F3F11F08F5F878BF601A8
:104940008789863010F186898F5F868B843158F491
:10495000858D41A16A2D8F700E94E539F601178A75
:1049600083E0878312C0F601858D41A16A2D8F7087
:104970000E94E539F60187858160878789818F5F8D
:104980000E945F2F02C0F601178AF601878580FF1B
:1049900005C080915C098F5F80935C09F601878573
:1049A00083FF05C080915A098F5F80935A09F601F1
:1049B00087858111B39489818F5F8983823208F45E
:1049C00089CD82C280912F04813009F0B0C1198253
:1049D0008981482F823208F077C2242F332785E25D
:1049E00090E0289FB001299F700D389F700D112411
:1049F000FB01EB5CFB4F87858F7D878785E2489FB6
:104A0000C00111240F2EF5E3CF2EF4E0DF2EF02DA0
:104A1000C80ED91EF601858D9927807F9070803A47
:104A2000910529F40F2EF1E4AF2EF02D0CC0F60104
:104A3000858D9927807F9070803B910521F40F2E02
:104A4000F2E4AF2EF02DF601848182FD4FC080810B
:104A500099278130910569F18034910509F046C0AC
:104A6000818199278F30910561F0803F9105F1F5A3
:104A7000858D41A16A2D8F700E949A398824839474
:104A800035C08981282F332785E290E0289FA00137
:104A9000299F500D389F500D1124FA01EB5CFB4FFC
:104AA000858DF60141A16A2D8F700E94E539882419
:104AB0001DC0F601818199278F30910561F0803FFB
:104AC0009105A1F4858D41A16A2D8F700E949A39BC
:104AD000882483940BC0F601858D41A16A2D8F70C7
:104AE0000E94E5398FE0F60181838824F6018181F7
:104AF000803F09F057C082A18F3F09F453C00E9444
:104B0000F1037C0100271127F601F4A2E3A28981B9
:104B10009927FC01E15EF64F80819927AA27BB27E0
:104B20008E159F05A007B10724F0EE24FF2487010E
:104B30000AC089819927FC01E15EF64F8081E81A5D
:104B4000F10801091109F3E0EF16F104010511055F
:104B5000CCF089819927880F991FFC01EF5CF64FF3
:104B6000808191819C0144275527C801B7010E948B
:104B7000326220EE31E040E050E00E94A66279010E
:104B80008A0103C0EE24FF248701F601F18AE08A3E
:104B900080915609909157098E0D9F1D909357094A
:104BA00080935609F6012089318982899389821779
:104BB000930788F5848185FF22C084899589892B94
:104BC00081F587858860878780915A098F5F8093F8
:104BD0005A098081813059F4858D41A16A2D8F70E9
:104BE0000E94E53988248FE0F601818382838981E0
:104BF000F601608971898F5F0E94272F12C0F6012C
:104C0000848180628483968185E0989FC00111240D
:104C1000958B848B06C0F60184818F7D8483158AF1
:104C2000148AF601868D9927807F9070803A9105CD
:104C300029F40F2EF1E49F2EF02D0CC0F601868D85
:104C40009927807F9070803B910521F40F2EF2E42C
:104C50009F2EF02DF601868D41A1692D8F700E9447
:104C6000683A282FF6018785992783FD42C080FD89
:104C700040C090915909809111018917D0F5F1E058
:104C80008F16A9F5222399F5F6018781882389F5E6
:104C90008485882371F58181803F59F587898F3F0D
:104CA00011F08F5F878BF6018789863010F1868936
:104CB0008F5F868B843158F4858D41A16A2D8F706A
:104CC0000E94E539F601178A83E0878312C0F60156
:104CD000858D41A16A2D8F700E94E539F601878587
:104CE0008160878789818F5F0E945F2F02C0F601F4
:104CF000178AF601878580FF05C080915C098F5F68
:104D000080935C09F601878583FF05C080915A096D
:104D10008F5F80935A09F60187858111B394898149
:104D20008F5F8983482F823208F457CECDC080919F
:104D30002F04823009F0C8C019828981982F8232ED
:104D400008F0C2C085E2989FC00111240F2EF5E340
:104D5000CF2EF4E0DF2EF02DC80ED91EF601858D82
:104D60009927807F9070803A910529F40F2EF1E405
:104D7000AF2EF02D0CC0F601858D9927807F9070A5
:104D8000803B910521F40F2EF2E4AF2EF02D4091DF
:104D900055094423D1F0898199279C012F5F3F4F0A
:104DA000842F99272817390741F4F601858D41A1F1
:104DB0006A2D8F700E949A390FC0F601858D41A12E
:104DC0006A2D8F700E94E53907C0F601858D41A1DB
:104DD0006A2D8F700E949A39F60182A18F3F09F4E3
:104DE0006CC00E94F1037C0100271127F601F4A298
:104DF000E3A280912E0480FF1CC089819927FC01C9
:104E0000E15EF64F80819927AA27BB278E159F0563
:104E1000A007B10724F0EE24FF2487010AC089818E
:104E20009927FC01E15EF64F8081E81AF10801093B
:104E30001109F3E0EF16F1040105110574F18091F9
:104E40002E0481FF19C089819927880F991FFC01C1
:104E5000EF5CF64F808191819C0144275527C80162
:104E6000B7010E94326220EE31E040E050E00E9443
:104E7000A66279018A0114C0C801B70128EB31E0AC
:104E800040E050E00E94326220EE31E040E050E02D
:104E90000E94A66279018A0103C0EE24FF248701E3
:104EA000F601F18AE08A80915609909157098E0D9A
:104EB0009F1D909357098093560989818F5F89833D
:104EC000982F823208F43ECFBB2031F4B0925B09B8
:104ED000B0925C09B0925D090E941605982F8093EC
:104EE000580980913004891710F490933004209170
:104EF00056093091570980913104909132048217FC
:104F0000930720F4309332042093310421960FB696
:104F1000F894DEBF0FBECDBFDF91CF911F910F91EF
:104F2000FF90EF90DF90CF90BF90AF909F908F90C9
:104F30000895815099270895CF93DF93EC01862F30
:104F40000E949927833278F4282F332785E290E056
:104F5000289FA001299F500D389F500D1124FA0160
:104F6000EB5CFB4FC683DF91CF910895EF92FF92E8
:104F70001F93CF937C01C0E080EC0E9425418111FA
:104F8000C1E081EC0E9425418111C26082EC0E9447
:104F900025418111C46081ED0E9425418111C860C5
:104FA00084EC0E9425418111C06185EC0E9425415D
:104FB0008111C06286EC0E9425418111C06487EC9A
:104FC0000E9425418111C06810E083EC0E942541B8
:104FD000811111E082ED0E9425418111126083ED63
:104FE0000E94254181111460F701C0831183C0E044
:104FF00081E00E94E7108111C1E082E00E94E71089
:105000008111C26083E00E94E7108111C46084E0D6
:105010000E94E7108111C86085E00E94E7108111AD
:10502000C06186E00E94E7108111C06287E00E94A3
:10503000E7108111C06488E00E94E7108111C06808
:10504000F701C283C0E089E00E94E7108111C1E04E
:105050008AE00E94E7108111C2608BE00E94E71095
:105060008111C4608CE00E94E7108111C8608DE05E
:105070000E94E7108111C0618EE00E94E71081114B
:10508000C0628FE00E94E7108111C06480E10E943D
:10509000E7108111C068F701C383C0E081E10E947D
:1050A000E7108111C1E082E10E94E7108111C26026
:1050B00083E10E94E7108111C46084E10E94E7103F
:1050C0008111C86085E10E94E7108111C06186E10D
:1050D0000E94E7108111C06287E10E94E7108111F0
:1050E000C06488E10E94E7108111C068F701C483A1
:1050F000C0E089E10E94E7108111C1E08AE10E94CD
:10510000E7108111C2608BE10E94E7108111C46039
:105110008CE10E94E7108111C8608DE10E94E710C8
:105120008111C0618EE10E94E7108111C0628FE1A0
:105130000E94E7108111C06480E20E94E710811193
:10514000C068F701C583CF911F91FF90EF9008953C
:105150001F93CF93DF93182FEB010E949927482FBD
:10516000833218F080E090E073C0992725E230E0A8
:10517000829FB001839F700D929F700D1124FB01DF
:10518000E75CFB4F208122FD24C0FB01EB5CFB4F61
:105190008181803F71F485859685892B39F421FDC5
:1051A00005C020FD03C0878585FF03C08FE088838D
:1051B00035C0242F332785E290E0289FF001299FF6
:1051C000F00D389FF00D1124EB5CFB4F818188833B
:1051D00025C030E0232F5EE0259FC0011124DC01B3
:1051E000A256B64FFD018181813099F490E07FE0B5
:1051F00060EFFD01E90FF11D8285841739F431E07C
:105200008C9182FF02C0788301C068839F5F9430D5
:1052100080F32F5F253010F43323F1F2242F33274E
:1052200085E290E0289FA001299F500D389F500DE6
:105230001124FA01EB5CFB4F878589838089918972
:105240009C838B83812F0E94AA2F8A8381E090E028
:10525000DF91CF911F9108950E949927833218F012
:1052600080E090E00895282F332785E290E0289F82
:10527000A001299F500D389F500D1124FA01EB5CBD
:10528000FB4F8181803F59F4FA01E75CFB4F20819D
:1052900021FD05C020FD03C081E090E0089580E07D
:1052A00090E008950E949927833218F080E090E002
:1052B0000895282F332785E290E0289FA001299F99
:1052C000500D389F500D1124FA01EB5CFB4F2785E0
:1052D000283011F0213019F481E090E0089580E049
:1052E00090E00895FC0180915609909157099183AF
:1052F00080838091580982838091590983838091AA
:105300005A09848380915B09858380915C09868337
:1053100080915D0987830895982F8150823238F4F7
:1053200085E2989FC0011124805F9B4F089580E023
:1053300090E008959EEF81B1892381B982B18923DC
:1053400082B917B818B891EF8AB189238AB98BB19D
:1053500089238BB908950F930E949927282F8331B1
:1053600068F000E0202F40E050E06BE27BE083E15A
:1053700091E00E94B42C80E090E007C08FE199E0BA
:10538000FC01E20FF11D808199270F9108950F9381
:105390000E949927833168F000E0202F40E050E020
:1053A00069E37BE083E191E00E94B42C80E692E225
:1053B00012C09927880F991FFC01EF5CF64F2081DE
:1053C000318184E190E0289FA001299F500D389FF2
:1053D000500D1124CA010F9108950F93CF93DF93BD
:1053E000EB010E949927833158F000E0202F40E024
:1053F00050E068E47BE083E191E00E94B42C12C0AD
:10540000992721E339E0880F991FFC01E20FF31F70
:10541000CE0164E170E00E945D6271836083C90126
:105420000E949332DF91CF910F9108950E949927A6
:10543000833118F080E090E00895282F332785E22B
:1054400090E0289FA001299F500D389F500D1124F6
:10545000FA01EB5CFB4F8089918908950E9499279E
:10546000833118F080E090E00895282F332785E2FB
:1054700090E0289FA001299F500D389F500D1124C6
:10548000FA01EB5CFB4F83A194A1089580932E0455
:105490006093550908951F93CF93C0E015E2C19F13
:1054A000C0011124FC01EB5CFB4F82A18F3F41F056
:1054B0000E94F1032C2F3327F901E15EF64F808320
:1054C000CF5FC23160F38FE199E00E947332CF91D8
:1054D0001F910895CF9380912F04833059F083E07A
:1054E00080932F04C0E061E08C2F0E94DE18CF5F14
:1054F000C232C8F3CF91089580919709882341F073
:105500000E94892A0E94B42A82E699E00E94012B17
:105510000895259A2D98269A2E988AEA80938000DD
:1055200089E180938100109285001092840080E3CD
:1055300095E09093870080938600109289001092E6
:10554000880010928B0010928A0010928D001092A9
:105550008C0060E070E081E00E94DF2A60E070E093
:1055600082E00E94DF2A08951092900084E08093E8
:105570009100109295001092940010929700109252
:105580009600109299001092980010929B00109231
:105590009A0010929D0010929C0010925F09109248
:1055A0005E0910926109109260098091690088601B
:1055B0008093690010926A00E99AE19A0895992708
:1055C0008230910581F0833091051CF4019721F020
:1055D0000895039779F00895872F9927809389007C
:1055E000609388000895872F992780938B0060939C
:1055F0008A000895872F992780938D0060938C00EF
:105600000895FC01118210821382128285E090E0DD
:105610009583848316820895EF92FF920F931F93D0
:10562000CF93DF93EC018E81982F8F5F8E8396301E
:1056300068F060E375E081E00E94DF2A60E375E0D6
:1056400082E00E94DF2A86E08E8355C08A819B819A
:105650009C0144275527888199817C0100271127C7
:10566000DA01C901689412F8880F991FAA1FBB1F9D
:105670001694D1F7820F931FA41FB51F280F391F4F
:105680004A1F5B1FCA01B90125E830E040E050E045
:105690000E943262A80197010E948462E901C90157
:1056A000845490408652944010F0C0E3D5E080913D
:1056B0009709882349F08091EF04803F29F4BE01C7
:1056C00081E00E94DF2A05C060E375E081E00E946E
:1056D000DF2A80919809882349F080911706803F3E
:1056E00029F4BE0182E00E94DF2A05C060E375E074
:1056F00082E00E94DF2ADF91CF911F910F91FF90EE
:10570000EF9008951F920F920FB60F9211242F93CE
:105710003F938F939F9380919400282F3327322FAC
:105720002227809195009927282B392B8091690099
:1057300099278C7090700C97E1F430936309209353
:105740006209109294001092950080913304909118
:105750003404909365098093640910923404109284
:10576000330410926809809169008B7F80936900EF
:1057700010C08091690099278C709070089749F447
:1057800030933404209333048091690084608093C3
:1057900069009F918F913F912F910F900FBE0F90B5
:1057A0001F901895CF93DF93CDB7DEB723970FB631
:1057B000F894DEBF0FBECDBFFE013196A0E8B1E088
:1057C00083E090E021E08030920719F40E940063AA
:1057D00003C0182E0E94006343E050E061E571E0D1
:1057E000CE0101960E942751882391F00E94122C2D
:1057F000E1E5F1E0A0E8B1E083E090E021E0803075
:10580000920719F40E94116303C0182E0E941163BD
:10581000279823960FB6F894DEBF0FBECDBFDF9159
:10582000CF910895CF93DF93CDB7DEB76E970FB6C4
:10583000F894DEBF0FBECDBF84E1FE013B9611920E
:105840008A95E9F740E064E124E130E0522FFE015F
:105850003B96469FC0011124DC01AC57BE4F211579
:10586000310551F081E02030380719F40E941163AE
:1058700003C0152E0E941163A8954F5F483038F37E
:105880001982FE013196A3E8B1E081E090E021E0C9
:105890008030920719F40E94116303C0182E0E94F1
:1058A00011636E960FB6F894DEBF0FBECDBFDF91C9
:1058B000CF910895CF93DF93CDB7DEB721970FB681
:1058C000F894DEBF0FBECDBFFE013196A3E8B1E074
:1058D00081E090E021E08030920719F40E9400639B
:1058E00003C0182E0E9400638981893010F088E07F
:1058F00089838981992721960FB6F894DEBF0FBE60
:10590000CDBFDF91CF910895CF93DF93CDB7DEB7B1
:1059100064970FB6F894DEBF0FBECDBF9B01FE01AA
:10592000319694E1899FD0011124A059BE4F84E1A2
:1059300090E041E08030940719F40E94006303C0B6
:10594000182E0E94006384E1FE013196D901019076
:105950000D928A95E1F764960FB6F894DEBF0FBEFC
:10596000CDBFDF91CF9108956F927F928F929F92DA
:10597000AF92BF92CF92DF92EF92FF920F931F935D
:10598000CF93DF93CDB7DEB7A9970FB6F894DEBFFC
:105990000FBECDBF6C015B013A01022FFE01B9962B
:1059A000A3E8B1E081E090E021E08030920719F4B3
:1059B0000E94006303C0182E0E94006389A58830EE
:1059C00008F0D4C09924FE01759684E1DF011D9290
:1059D0008A95E9F7B601CF010E942B62192D89A59E
:1059E000981608F05EC00F2EF4E18F2EF02D0F2ECA
:1059F000F4E1EF2EFF24F02DFE013196189DC00139
:105A00001124DC01AC57BE4FE114F10459F020E041
:105A1000E21621E0F20619F40E94006303C01E2C76
:105A20000E9400638D859E858A159B0599F546E049
:105A300050E0B601CE0101960E942751882351F50E
:105A4000992493948F858A3008F090C0890D8F87B0
:105A5000053008F004E0198A1A8A1B8A1C8A802FF4
:105A60009927AC01B301CE0141960E941462FE0158
:105A70003196189DD0011124AC57BE4F84E190E0BF
:105A800021E08030920719F40E94116303C0182EA0
:105A90000E9411631F5F89A5181718F4992009F453
:105AA000ABCF992009F052C089A5883008F04EC0CC
:105AB0008F5F89A78CE0FE01319611928A95E9F7F4
:105AC000F60101900020E9F731972E2F2C192C3088
:105AD00008F02BE010E0121780F4AE014F5F5F4F2B
:105AE000812F9927DC01A40FB51FF601E80FF91FDC
:105AF00080818C931F5F121798F3BE86AD8681E07C
:105B00008F87053008F004E0088B198A1A8A1B8AEF
:105B10001C8A802F9927AC01B301CE0141960E94C7
:105B20001462FE01319699A584E1989FD001112459
:105B3000A059BE4F84E190E021E08030920719F433
:105B40000E94116303C0182E0E941163FE01B996D2
:105B5000A3E8B1E081E090E021E08030920719F401
:105B60000E94116303C0182E0E941163A9960FB6FC
:105B7000F894DEBF0FBECDBFDF91CF911F910F9183
:105B8000FF90EF90DF90CF90BF90AF909F908F905D
:105B90007F906F900895089582E1E9E8FEE0119208
:105BA0008A95E9F780E1EBE9FEE011928A95E9F741
:105BB000EDEBFEE0A8E8B0E082E190E021E080308B
:105BC000920719F40E94006303C0182E0E9400631C
:105BD000EFECFEE0AAE9B0E082E190E021E0803065
:105BE000920719F40E94006303C0182E0E940063FC
:105BF000E1EEFEE0ACEAB0E080E190E021E0803050
:105C0000920719F40E94006303C0182E0E940063DB
:105C1000EBEAFEE0ADEBB0E082E190E021E0803025
:105C2000920719F40E94006303C0182E0E940063BB
:105C3000EAEEF9E0A5E8B0E081E090E021E0803014
:105C4000920719F40E94006303C0182E0E9400639B
:105C5000EBEEF9E0A6E8B0E082E090E021E08030F1
:105C6000920719F40E9400630895182E0E940063A1
:105C70000895CF93DF93CDB7DEB762970FB6F89450
:105C8000DEBF0FBECDBFFE01319682E1DF011D9266
:105C90008A95E9F7A8E8B0E082E190E021E0803061
:105CA000920719F40E94116303C0182E0E94116319
:105CB000FE013196AAE9B0E082E190E021E0803077
:105CC000920719F40E94116303C0182E0E941163F9
:105CD000FE013196ACEAB0E080E190E021E0803056
:105CE000920719F40E94116303C0182E0E941163D9
:105CF000FE013196ADEBB0E082E190E021E0803032
:105D0000920719F40E94116303C0182E0E941163B8
:105D10000E94CC2D62960FB6F894DEBF0FBECDBFA9
:105D2000DF91CF9108950E949F19982F8091EA09E1
:105D3000891790F49093EA09EAEEF9E0A5E8B0E05B
:105D400081E090E021E08030920719F40E94116315
:105D500003C0182E0E9411630E949A199C01809121
:105D6000EB099091EC0982179307A0F43093EC09AA
:105D70002093EB09EBEEF9E0A6E8B0E082E090E0DA
:105D800021E08030920719F40E9411630895182EC3
:105D90000E94116308958091EA09992708958091DE
:105DA000EB099091EC09089590E049E85EE0292F15
:105DB0003327F901E40FF51F808180FF17C08E7F24
:105DC0008083D901A857BF4FF901E354F14F808177
:105DD000082E0E940563D901A656BF4FF901E15371
:105DE000F14F8081082E0E9405630895E92FFF2757
:105DF000DF01A40FB51F8C9181FF0CC08D7F8C93A8
:105E0000DF01A354BF4FE555F14F8081082E0E945A
:105E1000056308959F5F923150F290E02BE93EE0D8
:105E2000E92FFF27DF01A20FB31F8C91813059F4B6
:105E30001C92DF01A455BF4FEF51F14F8081082E16
:105E40000E94056308959F5F903150F30895282FB5
:105E50002150223198F58DEB9EE0FC01E20FF11DFF
:105E60003081832F9927929582958F7089279F7013
:105E700089278F30910514F5482F4F5F942F929505
:105E8000907F832F8F70890F8083CB0183709070F8
:105E9000892B11F041E001C040E03327F901E153C3
:105EA000F14FCB019695879596958795840F8083C2
:105EB000F901E757F14F8081816080830895E82FD1
:105EC000E150E231C0F4FF27DF01A354B14F2C9120
:105ED000822F99278F7090700F971CF5822F8F70EB
:105EE0008F5F922F907F890F8C93E757F14F8081BE
:105EF0008160808308958351803198F4E82FFF27D3
:105F0000DF01AF51B14F2C91822F99278F70907084
:105F10000F973CF4822F8F5F8C93E556F14F81E011
:105F20008083089581508231A0F4E82FFF27DF019C
:105F3000A555B14F2C91822F99278F7090700F9794
:105F400044F4822F8F5F8C93E757F14F80818260FA
:105F500080830895E82FE150E23188F42E2F332713
:105F6000F901E354F14F8081882331F4F901E555BB
:105F7000F14F8081882391F081E090E00895282FEF
:105F80002351203158F481EE9EE0FC01E20FF11D17
:105F90008081882319F081E090E0089580E090E00E
:105FA0000895CF93DF93EC01FC0120E532E08EE011
:105FB00090E041E08030940721F4D9010E94116300
:105FC00004C0D901182E0E941163CE010296AC01C3
:105FD000698188810E94A319DF91CF910895FC0106
:105FE000A0E5B2E08EE090E021E08030920719F465
:105FF0000E9400630895182E0E9400630895FC011A
:10600000A0E6B2E08FE190E021E08030920719F441
:106010000E9411630895182E0E9411630895FC01D7
:10602000A0E6B2E08FE190E021E08030920719F421
:106030000E9400630895182E0E9400630895FC01D9
:10604000ACE7BBE088E090E021E08030920719F4F3
:106050000E9411630895182E0E9411630895FC0197
:10606000ACE7BBE088E090E021E08030920719F4D3
:106070000E9400630895182E0E94006308950F93F4
:10608000CF93DF93CDB7DEB721970FB6F894DEBF7D
:106090000FBECDBF8983853060F000E021E0AE0106
:1060A0004F5F5F4F67E470E085E591E00E94B42C9C
:1060B00015C0898199E1899FC0011124FB01DC0190
:1060C000A252B14F89E190E021E08030920719F4AB
:1060D0000E94116303C0182E0E94116321960FB60F
:1060E000F894DEBF0FBECDBFDF91CF910F91089521
:1060F0000F93CF93DF93CDB7DEB721970FB6F89408
:10610000DEBF0FBECDBF8983853060F000E021E0A7
:10611000AE014F5F5F4F64E570E085E591E00E945E
:10612000B42C15C0898199E1899FC0011124FB011C
:10613000DC01A252B14F89E190E021E0803092076A
:1061400019F40E94006303C0182E0E940063219678
:106150000FB6F894DEBF0FBECDBFDF91CF910F9188
:1061600008950F93CF93DF93CDB7DEB721970FB686
:10617000F894DEBF0FBECDBF8983803260F000E0AF
:1061800021E0AE014F5F5F4F60E670E085E591E092
:106190000E94B42C14C0FB0199818CE2989FD0011D
:1061A0001124A659BC4F8CE290E021E08030920788
:1061B00019F40E94116303C0182E0E9411632196E6
:1061C0000FB6F894DEBF0FBECDBFDF91CF910F9118
:1061D00008950F93CF93DF93CDB7DEB721970FB616
:1061E000F894DEBF0FBECDBF8983803260F000E03F
:1061F00021E0AE014F5F5F4F6AE670E085E591E018
:106200000E94B42C14C0FB0199818CE2989FD001AC
:106210001124A659BC4F8CE290E021E08030920717
:1062200019F40E94006303C0182E0E940063219697
:106230000FB6F894DEBF0FBECDBFDF91CF910F91A7
:1062400008950F93CF93DF93CDB7DEB721970FB6A5
:10625000F894DEBF0FBECDBF8983843160F000E0CB
:1062600021E0AE014F5F5F4F64E770E085E591E0AC
:106270000E94B42C14C0FB01998188E1989FD00141
:106280001124A451B74F88E190E021E080309207BB
:1062900019F40E94116303C0182E0E941163219605
:1062A0000FB6F894DEBF0FBECDBFDF91CF910F9137
:1062B00008950F93CF93DF93CDB7DEB721970FB635
:1062C000F894DEBF0FBECDBF8983843160F000E05B
:1062D00021E0AE014F5F5F4F6EE770E085E591E032
:1062E0000E94B42C14C0FB01998188E1989FD001D1
:1062F0001124A451B74F88E190E021E0803092074B
:1063000019F40E94006303C0182E0E9400632196B6
:106310000FB6F894DEBF0FBECDBFDF91CF910F91C6
:106320000895CF93DF93CDB7DEB769970FB6F89492
:10633000DEBF0FBECDBFFC01862F8150823218F028
:1063400080E090E02AC061508081898381818A83C6
:1063500082818B8383818C83878188878789888FDB
:10636000808D898F848195819E838D8386818F83A3
:10637000DF0118968FE0FE0139960D9001928A9503
:10638000E1F789E1689FC00111248457944FBC0153
:10639000CE0101960E946232992769960FB6F89451
:1063A000DEBF0FBECDBFDF91CF9108950F931F9336
:1063B000CF93DF93CDB7DEB769970FB6F894DEBF02
:1063C0000FBECDBF8C01962F91509232B0F589E16E
:1063D000989FC00111249E012F5F3F4FDC01A457FD
:1063E000B44F89E190E041E08030940721F4F90155
:1063F0000E94006304C0F901182E0E940063898185
:10640000F80180838A8181838B8182838C8183835D
:1064100088858783888D878B898D808F8D819E81EC
:10642000958384838F818683D80118968FE0FE013F
:10643000399601900D928A95E1F769960FB6F89416
:10644000DEBF0FBECDBFDF91CF911F910F91089599
:1064500081508B30C8F4FB01A82FBB27CD0182955A
:106460009295907F9827807F9827DC01A453B54FA1
:1064700080E190E021E08030920719F40E941163DE
:106480000895182E0E941163089581508B30C8F42E
:10649000FB01A82FBB27CD0182959295907F98276D
:1064A000807F9827DC01A453B54F80E190E021E084
:1064B0008030920719F40E9400630895182E0E94FC
:1064C00000630895FC01DB0189E190E021E0803068
:1064D000920719F40E94116303C0182E0E941163E1
:1064E00081E090E00895FC01A0E1B0E082E190E05D
:1064F00021E08030920719F40E9411630895182E4C
:106500000E9411630895FC01A0E1B0E082E190E0F7
:1065100021E08030920719F40E9400630895182E3C
:106520000E9400630895FC01A0E3B0E084E290E0E3
:1065300021E08030920719F40E9411630895182E0B
:106540000E9411630895FC01A0E3B0E084E290E0B2
:1065500021E08030920719F40E9400630895182EFC
:106560000E9400630895FC01A0E8B2E088E190E099
:1065700021E08030920719F40E9411630895182ECB
:106580000E9411630895FC01A0E8B2E088E190E068
:1065900021E08030920719F40E9400630895182EBC
:1065A0000E94006308950F93FC018081882319F4F1
:1065B00088E992E016C08081813019F48EED92E076
:1065C00010C08081823019F484E293E00AC000E0B8
:1065D00021E0AF0167E471E085E591E00E94B42C11
:1065E0000DC0DC0186E490E021E08030920719F4D0
:1065F0000E94116303C0182E0E9411630F91089529
:106600000F93CF93DF93CDB7DEB721970FB6F894F2
:10661000DEBF0FBECDBF8983882319F488E992E0DD
:1066200018C08981813019F48EED92E012C0898101
:10663000823019F484E293E00CC000E021E0AE0166
:106640004F5F5F4F60E671E085E591E00E94B42CFA
:106650000EC0FB01DC0186E490E021E0803092076F
:1066600019F40E94006303C0182E0E940063219653
:106670000FB6F894DEBF0FBECDBFDF91CF910F9163
:106680000895CF93DF93CDB7DEB760970FB6F89438
:10669000DEBF0FBECDBFFE013196A0E0B0E080E1CD
:1066A00090E021E08030920719F40E94006303C05B
:1066B000182E0E9400638B858F3119F48FE190E0D2
:1066C00008C08B85803219F480E290E002C08FE12F
:1066D00090E060960FB6F894DEBF0FBECDBFDF919D
:1066E000CF9108950F931F93CF93DF93CDB7DEB76C
:1066F0006E970FB6F894DEBF0FBECDBFFE01319688
:10670000A0E0B0E084E090E021E08030920719F44E
:106710000E94006303C0182E0E94006344E050E012
:1067200069E671E0CE0101960E942751882309F4A1
:106730004DC08E010F5F1F4F8EE1D8011D928A95CB
:10674000E9F785E0E9E6F1E0D80101900D928A953C
:10675000E1F71D821E821F82188619861A861B8603
:106760000E94B31CF801A0E0B0E080E190E021E0DD
:106770008030920719F40E94116303C0182E0E9402
:106780001163FE01319684E1DF011D928A95E9F7DC
:10679000AAEDBFE084E190E021E08030920719F497
:1067A0000E94116303C0182E0E941163FE013196EE
:1067B000A0E0B0E084E090E021E08030920719F49E
:1067C0000E94116303C0182E0E941163FE013196CE
:1067D000A0E3B2E08AE090E021E08030920719F473
:1067E0000E94006303C0182E0E9400634AE050E03C
:1067F00065E871E0CE0101960E942751882379F166
:106800000E94D31C0E947B100E94FA520E945506DF
:106810000E94FA0EFE0131968EE1DF011D928A95EB
:10682000E9F7AEE5BFE080E190E021E0803092073B
:1068300019F40E94116303C0182E0E941163E5E849
:10684000F1E0A0E3B2E08AE090E021E0803092073E
:1068500019F40E94116303C0182E0E941163FE01F7
:106860003196A0E8B1E083E090E021E0803092072B
:1068700019F40E94006303C0182E0E94006343E0D5
:1068800050E06EE671E0CE0101960E942751882308
:1068900091F00E94122CEEE6F1E0A0E8B1E083E076
:1068A00090E021E08030920719F40E94116303C048
:1068B000182E0E941163FE013196A0E8B0E085E039
:1068C00090E021E08030920719F40E94006303C039
:1068D000182E0E94006345E050E062E771E0CE01AF
:1068E00001960E942751882309F475C0FE01319654
:1068F0008EE1DF011D928A95E9F7ACEBB0E081E013
:1069000090E021E08030920719F40E94116303C0E7
:10691000182E0E941163FE013196A5E8B0E081E0D7
:1069200090E021E08030920719F40E94116303C0C7
:10693000182E0E941163FE013196A6E8B0E082E0B5
:1069400090E021E08030920719F40E94116303C0A7
:10695000182E0E941163FE013196A8E8B0E082E192
:1069600090E021E08030920719F40E94116303C087
:10697000182E0E941163FE013196ACEAB0E080E16E
:1069800090E021E08030920719F40E94116303C067
:10699000182E0E941163FE013196ADEBB0E082E14A
:1069A00090E021E08030920719F40E94116303C047
:1069B000182E0E941163E2E7F1E0A0E8B0E085E064
:1069C00090E021E08030920719F40E94116303C027
:1069D000182E0E941163FE013196AAEDBFE089E0F6
:1069E00090E021E08030920731F40E94006306C0FD
:1069F0000E94116330C0182E0E94006390E09E0137
:106A00002F5F3F4F8981181634F5AE014F5F5F4FFE
:106A1000F901E90FF11D808180538A3090F089E0FF
:106A2000F90111928A95E9F7F901AAEDBFE089E031
:106A300090E021E080309207D9F2182E0E94116375
:106A40000AC09F5F983038F49A01FA01E90FF11DEE
:106A500080811816ECF2FE013196A3EEBFE089E0CA
:106A600090E021E08030920731F40E94006306C07C
:106A70000E94116330C0182E0E94006390E09E01B6
:106A80002F5F3F4F8981181634F5AE014F5F5F4F7E
:106A9000F901E90FF11D808180538A3090F089E07F
:106AA000F90111928A95E9F7F901A3EEBFE089E0B7
:106AB00090E021E080309207D9F2182E0E941163F5
:106AC0000AC09F5F983038F49A01FA01E90FF11D6E
:106AD00080811816ECF26E960FB6F894DEBF0FBEEA
:106AE000CDBFDF91CF911F910F910895CFEFD0E1EE
:106AF000DEBFCDBF0E941A500E9494370E94C51974
:106B00000E9480050E942C500E946F420E94D22B4E
:106B10000E947233EBE6FEE0A0E7B0E08CE090E08C
:106B200021E08030920719F40E94006303C0182E00
:106B30000E94006380916B0E90916C0E8A3F9105CC
:106B400031F18B3F910538F48436910561F08D3732
:106B5000910599F039C021E0843F920711F1885ED8
:106B6000934049F131C086E28093E20084E0809353
:106B7000E30083E18093E40027C08EE18093E2008C
:106B800084E08093E30083E18093E4001DC08EE005
:106B90008093E20084E08093E30083E18093E4004B
:106BA00013C086E08093E20084E08093E30083E1F9
:106BB0008093E40009C082E08093E20084E0809347
:106BC000E30083E18093E4000E94300F80916D0E1A
:106BD00090916E0E059738F485E090E090936E0EDC
:106BE00080936D0E0DC080916D0E90916E0E815D43
:106BF000974030F080ED97E090936E0E80936D0E8D
:106C000080916F0E9091700E28E08030920738F0DE
:106C10008959994021F01092700E10926F0E0E94C7
:106C2000A63A0E94A9520E943B1E0E94B64187E0EC
:106C30000E94905C78940E94814EA89580E00E940A
:106C4000CB410E947A42FACF1F93162FA39899271F
:106C500087709070880F991F81640E942550812F42
:106C60000E94255080E00E942550A39A99271F91E9
:106C700008950F931F93162F042FA39899278770B9
:106C80009070880F991F80640E942550812F0E9468
:106C90002550802F0E942550A39A1F910F9108958F
:106CA0001F93CF93C091ED09CC2389F511E0109388
:106CB000ED094CE16AE08C2F0E9439364C2F6C2F85
:106CC0008C2F0E9439364FEF612F8C2F0E9439365E
:106CD0004C2F62E08C2F0E9439364C2F63E08C2FB2
:106CE0000E9439364C2F64E08C2F0E9439364C2F8D
:106CF00065E08C2F0E9439364C2F6CE08C2F0E945F
:106D000039364C2F6DE08C2F0E9439360AC1C09164
:106D1000ED09C13089F54CE16AE08C2F0E943936CB
:106D200040E0642F8C2F0E9439364FEF6C2F8C2F50
:106D30000E94393640E062E08C2F0E94393640E0F4
:106D400063E08C2F0E94393640E064E08C2F0E9473
:106D5000393640E065E08C2F0E94393640E06CE027
:106D60008C2F0E94393640E06DE08C2F0E9439361E
:106D700082E08093ED09D5C0C091ED09C23089F55C
:106D80004CE16AE08C2F0E94393640E0642F8C2F52
:106D90000E9439364FEF61E08C2F0E94393640E077
:106DA0006C2F8C2F0E94393640E063E08C2F0E94BC
:106DB000393640E064E08C2F0E94393640E065E0CF
:106DC0008C2F0E94393640E06CE08C2F0E943936BF
:106DD00040E06DE08C2F0E94393683E08093ED090E
:106DE000A0C0C091ED09C33089F54CE16AE08C2F59
:106DF0000E94393640E0642F8C2F0E9439364FEFC5
:106E000061E08C2F0E94393640E062E08C2F0E94B6
:106E1000393640E06C2F8C2F0E94393640E064E018
:106E20008C2F0E94393640E065E08C2F0E94393665
:106E300040E06CE08C2F0E94393640E06DE08C2FF2
:106E40000E94393684E08093ED096BC0C091ED0952
:106E5000C43089F54CE16AE08C2F0E9439364CEF42
:106E600060E08C2F0E9439364FEF61E08C2F0E943A
:106E7000393640E062E08C2F0E94393640E063E012
:106E80008C2F0E94393640E06C2F8C2F0E943936AF
:106E900040E065E08C2F0E94393640E06CE08C2F9A
:106EA0000E94393640E06DE08C2F0E94393685E033
:106EB0008093ED0936C0C091ED09C53081F54CE1F4
:106EC0006AE08C2F0E94393640E0642F8C2F0E949C
:106ED000393640EF61E08C2F0E94393640E062E0A5
:106EE0008C2F0E94393640E063E08C2F0E943936A7
:106EF00040E064E08C2F0E94393640E06C2F8C2FEC
:106F00000E94393640E06CE08C2F0E94393640E018
:106F10006DE08C2F0E9439361092ED0902C010925C
:106F2000ED09CF911F9108959B9AA39A4CE16AE0D5
:106F300080E00E94393640E064E1842F0E943936B7
:106F400040E0642F842F0E9439364FEF61E080E0EB
:106F50000E94393640E062E0842F0E94393640E0DA
:106F600063E0842F0E94393640E064E0842F0E9461
:106F7000393640E065E0842F0E94393640E06CE00D
:106F8000842F0E94393640E06DE0842F0E9439360C
:106F90004CE16AE081E00E94393640E064E181E042
:106FA0000E94393640E0642F81E00E9439364FEF6D
:106FB00061E0862F0E94393640E062E081E00E9465
:106FC000393640E063E081E00E94393640E064E019
:106FD00081E00E94393640E065E081E00E94393668
:106FE00040E06CE081E00E94393640E06DE081E0F5
:106FF0000E9439364CE16AE082E00E94393640E076
:1070000064E182E00E94393640E0642F82E00E9411
:1070100039364FEF61E082E00E94393640E062E0AD
:10702000862F0E94393640E063E082E00E943936C4
:1070300040E064E082E00E94393640E065E082E0B2
:107040000E94393640E06CE082E00E94393640E030
:107050006DE082E00E9439364CE16AE083E00E94F4
:10706000393640E064E183E00E94393640E0642F25
:1070700083E00E9439364FEF61E083E00E943936A9
:1070800040E062E083E00E94393640E063E0862F12
:107090000E94393640E064E083E00E94393640E0E7
:1070A00065E083E00E94393640E06CE083E00E94B6
:1070B000393640E06DE083E00E9439364CE16AE009
:1070C00084E00E94393640E064E184E00E94393671
:1070D0004CEF60E084E00E9439364FEF61E084E0DD
:1070E0000E94393640E062E084E00E94393640E098
:1070F00063E084E00E94393640E064E0862F0E941D
:10710000393640E065E084E00E94393640E06CE0CA
:1071100084E00E94393640E06DE084E00E94393618
:107120004CE16AE085E00E94393640E064E185E0A8
:107130000E94393640E065E185E00E94393640E042
:10714000642F85E00E94393640EF61E085E00E94BF
:10715000393640E062E085E00E94393640E063E085
:1071600085E00E94393640E064E085E00E943936CF
:1071700040E065E0862F0E94393640E06CE085E013
:107180000E94393640E06DE085E00E94393608956E
:107190000F931F93CF93082FC62F142F20E030E0BA
:1071A000613611F421E030E080E090E0C13411F468
:1071B00081E090E0822B932B892B91F060E0812F6E
:1071C0000E94243621E030E0002E02C0220F331F3F
:1071D0000A94E2F7482F422B60E0812F0E94393653
:1071E00020E030E0C23611F421E030E080E090E0B1
:1071F000C23411F481E090E0822B932B892B89F02B
:1072000061E0812F0E94243621E030E002C0220F8D
:10721000331F0A95E2F7482F422B61E0812F0E942D
:107220003936CF911F910F9108950F931F93CF93EC
:10723000082FC62F142F20E030E0613611F421E032
:1072400030E080E090E0C13411F481E090E0822BE6
:10725000932B892BA1F060E0812F0E94243621E03E
:1072600030E0002E02C0220F331F0A94E2F7922F63
:107270009095482F492360E0812F0E94393620E005
:1072800030E0C23611F421E030E080E090E0C2341A
:1072900011F481E090E0822B932B892B99F061E02F
:1072A000812F0E94243621E030E002C0220F331FDC
:1072B0000A95E2F7922F9095482F492361E0812F9C
:1072C0000E943936CF911F910F9108950F931F930C
:1072D000CF93182FC62F042F20E030E0613611F431
:1072E00021E030E080E090E0C13411F481E090E0F2
:1072F000822B932B892B29F0412F64E1802F0E9450
:10730000393620E030E0C23611F421E030E080E090
:1073100090E0C23411F481E090E0822B932B892B12
:1073200029F0412F65E1802F0E943936CF911F91BE
:107330000F9108950F931F93CF93082FC62F142FEB
:1073400050E020E030E0613611F421E030E080E0F0
:1073500090E0C13411F481E090E0822B932B892BD3
:1073600071F062E1812F0E94243621E030E0002E8E
:1073700002C0220F331F0A94E2F7582F522B20E04D
:1073800030E0C23611F421E030E080E090E0C23419
:1073900011F481E090E0822B932B892B69F063E15B
:1073A000812F0E94243621E030E002C0220F331FDB
:1073B0000A95E2F7582F522B412F6C2F852F0E94F0
:1073C0006639CF911F910F9108950F931F93CF931B
:1073D000082FC62F142F50E020E030E0613611F462
:1073E00021E030E080E090E0C13411F481E090E0F1
:1073F000822B932B892B81F062E1812F0E9424360E
:1074000021E030E0002E02C0220F331F0A94E2F781
:10741000922F9095582F592320E030E0C23611F476
:1074200021E030E080E090E0C23411F481E090E0AF
:10743000822B932B892B79F063E1812F0E942436D4
:1074400021E030E002C0220F331F0A95E2F7922FAD
:107450009095582F5923412F6C2F852F0E94663904
:10746000CF911F910F9108951F93CF93C82F162F7F
:1074700040E020E030E0813611F421E030E080E0AF
:1074800090E0C13411F481E090E0822B932B892BA2
:1074900029F062E1812F0E942436482F20E030E05D
:1074A000C23611F421E030E080E090E0C23411F403
:1074B00081E090E0822B932B892B29F063E1812FCF
:1074C0000E942436482F842F9927CF911F91089529
:1074D0000F931F93CF93182FC62F042F40E020E067
:1074E00030E0613611F421E030E080E090E0C1341A
:1074F00011F481E090E0822B932B892B29F062E13B
:10750000802F0E942436482F20E030E0C23611F44C
:1075100021E030E080E090E0C23411F481E090E0BE
:10752000822B932B892B29F063E1802F0E94243634
:10753000482F81E090E002C0880F991F1A95E2F76A
:1075400084239927CF911F910F9108950E94D21300
:107550008BE49AE09093E20A8093E10A1092E30AA6
:107560001092DA0A1092DB0A8AED9AE00E94DA138E
:107570008823D1F71092D90A83E59AE09093EE0A16
:107580008093ED0A1092EF0A1092E60A1092E70A31
:1075900086EE9AE00E94DA138823D1F71092E50A6A
:1075A0008BE59AE09093FA0A8093F90A1092FB0A0D
:1075B0001092F20A1092F30A82EF9AE00E94DA1314
:1075C0008823D1F71092F10A83E69AE09093060B94
:1075D0008093050B1092070B1092FE0A1092FF0A7F
:1075E0008EEF9AE00E94DA138823D1F71092FD0AF9
:1075F0008BEF99E09093730A8093720A1092740A49
:1076000010926B0A82E080936C0A8BE69AE00E94EB
:10761000DA138823D1F783E09AE090937E0A80936F
:107620007D0A10927F0A1092760A82E08093770A90
:1076300086E79AE00E94DA138823D1F78BE09AE07C
:107640009093890A8093880A10928A0A1092810A7C
:1076500082E08093820A81E89AE00E94DA1388230C
:10766000D1F783E19AE09093940A8093930A109261
:10767000950A10928C0A82E080938D0A8CE89AE039
:107680000E94DA138823D1F78BE19AE090939F0A46
:1076900080939E0A1092A00A1092970A82E080932B
:1076A000980A87E99AE00E94DA138823D1F783E2E7
:1076B0009AE09093AA0A8093A90A1092AB0A1092BA
:1076C000A20A82E08093A30A82EA9AE00E94DA1377
:1076D0008823D1F78BE29AE09093B50A8093B40A9D
:1076E0001092B60A1092AD0A82E08093AE0A8DEA3B
:1076F0009AE00E94DA138823D1F783E39AE090930B
:10770000C00A8093BF0A1092C10A1092B80A82E0A0
:107710008093B90A88EB9AE00E94DA138823D1F7A4
:107720008BE39AE09093CB0A8093CA0A1092CC0A1A
:107730001092C30A82E08093C40A83EC9AE00E940C
:10774000DA138823D1F783E49AE09093D60A8093E2
:10775000D50A1092D70A1092CE0A82E08093CF0AFF
:107760008EEC9AE00E94DA138823D1F70895809175
:10777000D90A8823E1F08091D90A813059F489ED42
:107780009AE001960E94DA13882389F482E08093BC
:10779000D90A0DC08091D90A823049F489ED9AE066
:1077A00001960E94EC14882311F48093D90A8091E9
:1077B000E50A8823E1F08091E50A813059F485EEED
:1077C0009AE001960E94DA13882389F482E080937C
:1077D000E50A0DC08091E50A823049F485EE9AE011
:1077E00001960E94EC14882311F48093E50A80919D
:1077F000F10A8823E1F08091F10A813059F481EF98
:107800009AE001960E94DA13882389F482E080933B
:10781000F10A0DC08091F10A823049F481EF9AE0BB
:1078200001960E94EC14882311F48093F10A809150
:10783000FD0A8823E1F08091FD0A813059F48DEF33
:107840009AE001960E94DA13882389F482E08093FB
:10785000FD0A08958091FD0A823049F48DEF9AE087
:1078600001960E94EC14882311F48093FD0A089578
:10787000CF93DF93EC018BE69AE00E94EC1488230F
:1078800009F046C080916D0A90916E0AAA27BB2725
:1078900088839983AA83BB83E091720AF091730A6B
:1078A00080818D83E091720AF091730A81818E83C9
:1078B000E091720AF091730A82818F83E091720ADB
:1078C000F091730A83818887E091720AF091730ABC
:1078D00084818987E091720AF091730A85818A8791
:1078E000E091720AF091730A86818B87E091720AA7
:1078F000F091730A87818C878091710A8C838BE663
:107900009AE00E94DA138823D1F781E090E0BBC2AD
:1079100086E79AE00E94EC14882309F046C0809123
:10792000780A9091790AAA27BB2788839983AA832A
:10793000BB83E0917D0AF0917E0A80818D83E09186
:107940007D0AF0917E0A81818E83E0917D0AF0911B
:107950007E0A82818F83E0917D0AF0917E0A838185
:107960008887E0917D0AF0917E0A84818987E09181
:107970007D0AF0917E0A85818A87E0917D0AF091E7
:107980007E0A86818B87E0917D0AF0917E0A87814D
:107990008C8780917C0A8C8386E79AE00E94DA13B8
:1079A0008823D1F781E090E06EC281E89AE00E94DE
:1079B000EC14882309F046C08091830A9091840AD0
:1079C000AA27BB2788839983AA83BB83E091880A6F
:1079D000F091890A80818D83E091880AF091890A6B
:1079E00081818E83E091880AF091890A82818F8358
:1079F000E091880AF091890A83818887E091880A5A
:107A0000F091890A84818987E091880AF091890A36
:107A100085818A87E091880AF091890A86818B871F
:107A2000E091880AF091890A87818C878091870A82
:107A30008C8381E89AE00E94DA138823D1F781E0F1
:107A400090E021C28CE89AE00E94EC14882309F0AF
:107A500046C080918E0A90918F0AAA27BB278883FF
:107A60009983AA83BB83E091930AF091940A808161
:107A70008D83E091930AF091940A81818E83E09145
:107A8000930AF091940A82818F83E091930AF09196
:107A9000940A83818887E091930AF091940A848103
:107AA0008987E091930AF091940A85818A87E09111
:107AB000930AF091940A86818B87E091930AF09162
:107AC000940A87818C878091920A8C838CE89AE053
:107AD0000E94DA138823D1F781E090E0D4C187E9CE
:107AE0009AE00E94EC14882309F046C08091990A1C
:107AF00090919A0AAA27BB2788839983AA83BB837C
:107B0000E0919E0AF0919F0A80818D83E0919E0A08
:107B1000F0919F0A81818E83E0919E0AF0919F0AE5
:107B200082818F83E0919E0AF0919F0A83818887EA
:107B3000E0919E0AF0919F0A84818987E0919E0AD4
:107B4000F0919F0A85818A87E0919E0AF0919F0AB1
:107B500086818B87E0919E0AF0919F0A87818C87AE
:107B600080919D0A8C8387E99AE00E94DA1388232A
:107B7000D1F781E090E087C182EA9AE00E94EC149C
:107B8000882309F046C08091A40A9091A50AAA27EB
:107B9000BB2788839983AA83BB83E091A90AF091CC
:107BA000AA0A80818D83E091A90AF091AA0A8181B5
:107BB0008E83E091A90AF091AA0A82818F83E091D5
:107BC000A90AF091AA0A83818887E091A90AF09115
:107BD000AA0A84818987E091A90AF091AA0A85817D
:107BE0008A87E091A90AF091AA0A86818B87E091A1
:107BF000A90AF091AA0A87818C878091A80A8C83B0
:107C000082EA9AE00E94DA138823D1F781E090E0BB
:107C10003AC18DEA9AE00E94EC14882309F046C02C
:107C20008091AF0A9091B00AAA27BB2788839983D5
:107C3000AA83BB83E091B40AF091B50A80818D8359
:107C4000E091B40AF091B50A81818E83E091B40A83
:107C5000F091B50A82818F83E091B40AF091B50A60
:107C600083818887E091B40AF091B50A848189877D
:107C7000E091B40AF091B50A85818A87E091B40A4F
:107C8000F091B50A86818B87E091B40AF091B50A2C
:107C900087818C878091B30A8C838DEA9AE00E9459
:107CA000DA138823D1F781E090E0EDC088EB9AE009
:107CB0000E94EC14882309F046C08091BA0A909182
:107CC000BB0AAA27BB2788839983AA83BB83E09139
:107CD000BF0AF091C00A80818D83E091BF0AF091C4
:107CE000C00A81818E83E091BF0AF091C00A82812F
:107CF0008F83E091BF0AF091C00A83818887E09169
:107D0000BF0AF091C00A84818987E091BF0AF0918F
:107D1000C00A85818A87E091BF0AF091C00A8681F6
:107D20008B87E091BF0AF091C00A87818C87809190
:107D3000BE0A8C8388EB9AE00E94DA138823D1F77D
:107D400081E090E0A0C083EC9AE00E94EC148823CC
:107D500009F046C08091C50A9091C60AAA27BB27A0
:107D600088839983AA83BB83E091CA0AF091CB0AE6
:107D700080818D83E091CA0AF091CB0A81818E8344
:107D8000E091CA0AF091CB0A82818F83E091CA0AFE
:107D9000F091CB0A83818887E091CA0AF091CB0ADF
:107DA00084818987E091CA0AF091CB0A85818A870C
:107DB000E091CA0AF091CB0A86818B87E091CA0ACA
:107DC000F091CB0A87818C878091C90A8C8383ECE0
:107DD0009AE00E94DA138823D1F781E090E053C043
:107DE0008EEC9AE00E94EC14882309F046C0809142
:107DF000D00A9091D10AAA27BB2788839983AA83A6
:107E0000BB83E091D50AF091D60A80818D83E09101
:107E1000D50AF091D60A81818E83E091D50AF0913E
:107E2000D60A82818F83E091D50AF091D60A8381A8
:107E30008887E091D50AF091D60A84818987E091FC
:107E4000D50AF091D60A85818A87E091D50AF0910A
:107E5000D60A86818B87E091D50AF091D60A878170
:107E60008C878091D40A8C838EEC9AE00E94DA137E
:107E70008823D1F781E090E006C0188219821A8227
:107E80001B8280E090E0DF91CF910895CF93DF9344
:107E9000DC018091D90A882339F489ED9AE0909326
:107EA0000A0B8093090B21C08091E50A882339F4DD
:107EB00085EE9AE090930A0B8093090B16C080918F
:107EC000F10A882339F481EF9AE090930A0B8093AA
:107ED000090B0BC08091FD0A882309F072C08DEF59
:107EE0009AE090930A0B8093090BE091090BF091B3
:107EF0000A0B0084F185E02DED018D818083E091F6
:107F0000090BF0910A0B0084F185E02D8E818183AD
:107F1000E091090BF0910A0B0084F185E02D8F812F
:107F20008283E091090BF0910A0B0084F185E02D2A
:107F300088858383E091090BF0910A0B0084F18519
:107F4000E02D89858483E091090BF0910A0B008470
:107F5000F185E02D8A858583E091090BF0910A0B6C
:107F60000084F185E02D8B858683E091090BF091EB
:107F70000A0B0084F185E02D8C858783E091090B45
:107F8000F0910A0B8C818783E091090BF0910A0B29
:107F90008D919C9194838383E091090BF0910A0B5E
:107FA0001286E091090BF0910A0B1182E091090B06
:107FB000F0910A0B1282E091090BF0910A0B81E01B
:107FC0008083DF91CF9108958EEE99E00E94383C36
:107FD000882361F18EEE99E00E9478118EEE99E08F
:107FE0000E94383C882311F18EEE99E00E947811AE
:107FF0008EEE99E00E94383C8823C1F08EEE99E025
:108000000E9478118EEE99E00E94383C882371F02E
:108010008EEE99E00E9478118EEE99E00E94383C35
:10802000882321F08EEE99E00E9478110895FF9246
:108030000F931F93CF93DF93CDB7DEB760970FB643
:10804000F894DEBF0FBECDBF20E0822F99278C01B0
:10805000055F144FF80180818C7F8083F22EF394AA
:10806000BE016F5F7F4F8F2D0E94453288898170DE
:10807000982F990F990F990FF80180818370892BA0
:1080800080832F2D2B3008F360960FB6F894DEBF57
:108090000FBECDBFDF91CF911F910F91FF9008953B
:1080A000FC01808183709927009719F0019731F0C6
:1080B000089580818D728162808308959081892FD7
:1080C000807FA1F493FD05C0892F8E7F8660808319
:1080D0000895808182FF03C08B7F808303C08081ED
:1080E0008460808380818C7F826080830895FC011E
:1080F00080818370992781309105BCF08330910590
:108100001CF0039731F0089580818F708362808323
:1081100008959081892F807F41F4892F8C7F8083FF
:1081200093FD03C0892F887F8083089530E0832FDB
:108130009927FC01E55FF44F2081822F807F41F079
:10814000822F807F982F9051822F8F70892B808370
:108150003F5F3B3060F3EBE0FBE0309B04C0CF01BE
:108160000E94504003C0CF010E947740ECE0FBE04A
:10817000319904C0CF010E94504003C0CF010E943A
:108180007740EDE0FBE0329904C0CF010E945040FF
:1081900003C0CF010E947740EEE0FBE0499904C0A4
:1081A000CF010E94504003C0CF010E947740EFE012
:1081B000FBE0349904C0CF010E94504003C0CF01BE
:1081C0000E947740E0E1FBE0359904C0CF010E94B6
:1081D000504003C0CF010E947740E1E1FBE03699B7
:1081E00004C0CF010E94504003C0CF010E947740DD
:1081F000E2E1FBE0379904C0CF010E94504003C088
:10820000CF010E947740E3E1FBE0339904C0CF0146
:108210000E94504003C0CF010E947740E4E1FBE0A0
:108220004A9904C0CF010E94504003C0CF010E9470
:108230007740E5E1FBE04B9904C0CF010E9450403C
:108240000895CF010E94774008959927853C9105B4
:1082500009F451C0863C9105ACF4823C9105B1F122
:10826000833C91053CF4803C910511F1813C9105E2
:1082700031F16BC0833C910509F452C0843C9105F7
:1082800099F163C0813D910541F1823D91053CF436
:10829000863C9105B9F1873C9105D9F156C0823DE4
:1082A000910509F444C0833D910509F447C04DC0D0
:1082B00080910B0B86958695817099270895809102
:1082C0000C0B8695869581709927089580910D0BEA
:1082D0008695869581709927089580910E0B8695D5
:1082E000869581709927089580910F0B86958695C4
:1082F0008170992708958091100B869586958170DD
:10830000992708958091110B8695869581709927FC
:1083100008958091120B869586958170992708950E
:108320008091130B86958695817099270895809189
:10833000140B869586958170992708958091150B69
:10834000869586958170992708958EEF90E008951F
:108350001092B60087E08093B0001092B2008EE4D5
:108360008093B30082E08093700008950E94A8413A
:108370001092180B1092190B10921A0B10921B0BE3
:108380001092200B1092210B0E9417400E94FE05B4
:108390000E94CC2D0895CF93C82F8091160B88236F
:1083A00011F01092160BA8950E94E43FC23011F014
:1083B0000E94B73BC23009F46FC08091170B88232D
:1083C00009F444C08091170B81508093170B809162
:1083D000180B8F5F8093180B823040F01092180BAF
:1083E0000E9496400E949D150E9438078091190BAB
:1083F0008F5F8093190B843040F01092190B0E940C
:1084000012160E942E530E94395080911A0B8F5FD2
:1084100080931A0B8A3030F010921A0BC13011F091
:108420000E94601180911B0B8F5F80931B0B843126
:1084300068F010921B0B8091200B8F5F8093200BB4
:108440000E9450360E943A170E9415118091200B0D
:108450008A3010F11092200B80911C0B90911D0B13
:10846000A0911E0BB0911F0B0196A11DB11D809311
:108470001C0B90931D0BA0931E0BB0931F0B0E941F
:10848000D42E8091210B8F5F8093210B8C3320F0B1
:108490001092210B0E94932ECF91089580911C0B76
:1084A00090911D0BA0911E0BB0911F0BBC01CD0133
:1084B00008951F920F920FB60F9211248F9310926E
:1084C000B20081E08093160B8091170B8F5F809331
:1084D000170B8F910F900FBE0F901F9018950E9451
:1084E000D84E0E948B5060E076E980E090E00E94D8
:1084F000A650089504C00E941E4F0E94714F0E9412
:10850000084F8823C1F70895FC0190E061506F3F48
:1085100021F0819198276150E0F7892F99270895DC
:108520000F931F938C01FC0181818150682FC8013A
:1085300001960E948442F801808381819927BC01C1
:10854000C8010E94394F1F910F910895AF92BF92B9
:10855000CF92DF92EF92FF920F931F93CF93DF930F
:10856000CDB7DEB7C35ED0400FB6F894DEBF0FBE06
:10857000CDBF6C01FC0181818150682FC60101963D
:108580000E948442D6019C91981711F00C94664E7B
:10859000F6018281882309F0F8C08381992781350B
:1085A000910509F449C0823591053CF48033910569
:1085B00089F08035910561F1E8C08335910509F4B2
:1085C0008EC0833591050CF478C08435910509F48B
:1085D000B2C0DBC08E01035D1F4F80E5D8011D9244
:1085E0008A95E9F785E18EA71FA680E888ABF6019A
:1085F000848189AB992796012B5F3F4FAC01B9016C
:10860000CE01C2960E941462C8010E949042BDC071
:108610008E01035D1F4F80E5D8011D928A95E9F711
:1086200085E08EA71FA680EA88AB0E945A2C89ABF2
:10863000C8010E949042A9C0F601B4800F2EFDE24D
:10864000EF2EFF24F02DEC0EFD1E80E5D7011D92CC
:108650008A95E9F789E18EA71FA681EA88AB8E018A
:1086600003581F4FB8018B2D0E94842CB9AA8CE0AF
:10867000FE01F296D8010D9001928A95E1F7F8017A
:10868000848595859FAF8EAF8685FE01E05CFF4FA8
:108690008083F8018785FE01EF5BFF4F8083992778
:1086A000AC01BE0163577F4FCE018E5B9F4F0E948E
:1086B0001462C7010E94904268C00E94122CFE0101
:1086C000BD9680E5DF011D928A95E9F784E08EA7CB
:1086D0001FA682EA88ABCF010E94904256C0F601E5
:1086E000458156818481FE01ED51FF4F80838131A8
:1086F00008F04BC080E5FE01BD9611928A95E9F71E
:1087000087E18EA71FA683EA88AB5BAB4AABFE016D
:10871000ED51FF4F808189ABFE01F4969927DA0174
:10872000019724F00E94F8620192FACFCE018D9653
:108730000E9490422AC0F601458156818481FE0143
:10874000ED51FF4F8083813100F5F601379699276F
:10875000DA01019724F001900E940563FACFDE014F
:108760009D9680E5FD0111928A95E9F787E08EA735
:108770001FA684EA88AB5BAB4AABFE01ED51FF4F0D
:10878000808189ABCD010E949042F60182818130C7
:1087900011F00C946F4E83819927AA27BB27FC0107
:1087A0003197EB36F10510F00C94584EE65BFF4F15
:1087B000EE0FFF1F0590F491E02D09940E946A2AA4
:1087C000F601B4808B2D8150823210F00C946F4EE4
:1087D00020E0AE01475F5F4F822F9927DA01A80F93
:1087E000B91FF601E80FF91F82858C932F5F2F3098
:1087F00098F3F6018581898386818A8387818B83BB
:10880000838D948D9E838D83858D8F8380858887CE
:1088100081858C83818D888F828D898F6B2DCE0190
:1088200001960E9491316B2DCE0101960E942D1F61
:108830001DA685E08EA711E01FA781E888AB19AAC5
:10884000CE018D960E949042812F0E94CB410C94C4
:108850006F4EF601B4808B2D8150823208F047C0F4
:108860006B2DCE0101960E94D6318EE18EA781E05C
:108870008FA782E888ABB9AA89818AAB8A818BAB42
:108880008B818CAB8C818EAB8D819E81FE01E85BF0
:10889000FF4F918380838F81FE01E65BFF4F8083D2
:1088A00020E0BE016F5F7F4FAE01475F5F4F822FB9
:1088B0009927DC01A60FB71FFA01E80FF91F808185
:1088C000FD0186AB2F5F2F3090F388858DAB888DAF
:1088D000FE01EA5BFF4F8083898DFE01E95BFF4F5C
:1088E0008083CE018D960E9490420C946F4EFFEFD4
:1088F000BF1611F00C946F4EFE01ED51FF4F108228
:10890000FE01ED51FF4F8081982F823210F00C94C0
:108910006F4E0F2EF3EEEF2EFF24F02DEC0EFD1E0A
:108920006E010894C11CD11C8E01075F1F4F892F57
:108930008F5F682FCE0101960E94D6318EE18EA7FF
:1089400081E08FA782E888ABD7018C918F5F89ABDC
:1089500089818AAB8A818BAB8B818CAB8C818EAB0E
:108960008D819E81FE01E85BFF4F918380838F8123
:10897000FE01E65BFF4F808320E0822F9927DC0118
:10898000AC0DBD1DF801E80FF91F8081FD0186AB1C
:108990002F5F2F3090F388858DAB888DFE01EA5BC9
:1089A000FF4F8083898DFE01E95BFF4F8083CE01FD
:1089B0008D960E94904281E00E94CB41D7018C911C
:1089C0008F5F8C93982F823208F4B1CF0C946F4E46
:1089D0000E946A2AF601B480AE0143585F4F9601A7
:1089E0002B5F3F4F8FE0DA01F90101900D928A95DC
:1089F000E1F7F6018489FA018787BA018B2D0E947D
:108A0000283281E08FA783E888ABB9AA85E08EA7DA
:108A1000CE018D960E9490420C946F4EF601B48068
:108A20008B2D81508A3010F581E08FA784E888ABC8
:108A3000B9AA8E0103581F4FB8018B2D0E944532F1
:108A40008FE0FE01F296D8010D9001928A95E1F730
:108A5000F8018785FE01EF5BFF4F808385E18EA7DC
:108A6000CE018D960E9490420C946F4EFFEFBF1680
:108A700011F00C946F4EFE01ED51FF4F1082FE017C
:108A8000ED51FF4F8081982F8B3010F00C946F4E7A
:108A9000BB24B3948E0103581F4F0F2EFFE0AF2E5F
:108AA000F02D0F2EF1E4EF2EFF24F02DEC0EFD1E25
:108AB0000F2EF3EECF2EDD24F02DCC0EDD1EBFA643
:108AC00084E888AB892F8F5F89ABB8010E9445325B
:108AD000FE01F296D8012A2D0D9001922A95E1F718
:108AE000F8018785D7018C9385E18EA7CE018D96FD
:108AF0000E9490428B2D0E94CB41F60180818F5FB6
:108B00008083982F8B30D8F20C946F4E0E946A2A83
:108B10000E94C519A8950E94D31CA8950E943B1ECF
:108B2000A8950E947B10A8950E94FA52A8950E94D1
:108B30005506A8950E94392E0E94FA0E81E08FA753
:108B400086E888AB84E08EA7CE018D960E94904285
:108B50000C946F4E84E18EA781E08FA787E888ABE5
:108B60008DE0A8E7B1E0FE01F1960D9001928A95A3
:108B7000E1F70E944E429B01AC01AA27BB278EAFB2
:108B8000BB27A52F942F832F8FAFFE01E05CFF4FF3
:108B90002083CE018D960E9490420C946F4E0C94CF
:108BA00000000C946F4EC60104960E941F3081E0B5
:108BB0008FA789E888AB84E08EA7CE018D960E94AE
:108BC00090420C946F4E81E08FA78AE888AB8CE0CE
:108BD0008EA7CE01C1960E942F30CE018D960E94A5
:108BE00090420C946F4ECE0187960E94B62781E08A
:108BF0008FA781EA88AB8FA189AB88A58AAB89A5AD
:108C00008BAB8AA58CAB8BA58DAB8CA58EAB8AE08C
:108C10008EA7CE018D960E9490420C946F4EF60165
:108C2000B480F1E2FB1500F1BE016E5D7F4F8B2D2C
:108C30000E94A82881E08FA782EA88ABB9AA8BA1FD
:108C40008BAB8CA18EAB8AA18AAB8DA19EA1892F03
:108C500099278CAB8DA18DAB8AE08EA7CE018D9626
:108C60000E9490420C946F4E2FEFB21611F00C94AC
:108C70006F4EFE01ED51FF4F1082FE01ED51FF4F8F
:108C80008081982F823210F00C946F4EFF24F39461
:108C90008F01BE016E5D7F4F892F8F5F0E94A828D4
:108CA000FFA682EA88ABD8018C918F5F89AB8BA13C
:108CB0008BAB8CA18EAB8AA18AAB8DA19EA1892F93
:108CC00099278CAB8DA18DAB8AE08EA7CE018D96B6
:108CD0000E9490428F2D0E94CB41F80180818F5FCE
:108CE0008083982F8232A8F20C946F4ECE014A9660
:108CF0000E9472298AE08EA781E08FA780EA88AB64
:108D000088A189AB8E8D8AAB8A8D9B8D892F9927FF
:108D10008BAB8A8D8CAB8D8D8DAB8C8D8EABCE015C
:108D20008D960E949042DBC7F601648180E00E942C
:108D3000E92184E08EA781E08FA783EA88ABCE018A
:108D40008D960E949042CBC7DE01A353BF4FF60120
:108D500084818C938581FD018183F6018681FD01EB
:108D60008283F6018781FD018383F6018085FD0101
:108D70008483F6018185FD018583F6018285FD01ED
:108D80008683F6018385FD018783CD010E94F12151
:108D900084E08EA781E08FA784EA88ABCE018D9610
:108DA0000E9490429CC7FE01E358FF4FA0E0B0E054
:108DB00080E190E021E08030920719F40E94006386
:108DC00003C0182E0E940063F60184819581A6815C
:108DD000B781FE01EF57FF4F80839183A283B38356
:108DE000DE01A358BF4FF6018085FD018087F601A3
:108DF0008185FD018187F6018285FD018287A0E0E2
:108E0000B0E080E190E021E08030920719F40E9408
:108E1000116303C0182E0E94116384E08EA781E0C5
:108E20008FA780EC88ABCE018D960E94904257C7E9
:108E3000FE01E358FF4FA0E0B0E080E190E021E0C8
:108E40008030920719F40E94006303C0182E0E941C
:108E500000638BE08EA781E08FA781EC88ABFE01D9
:108E6000EF57FF4F80819181A281B38189AB9AAB8B
:108E7000ABABBCABFE01E358FF4F80858DAB81856A
:108E80008EAB82858FABCE018D960E94904227C714
:108E90008AE38EA781E08FA780ED88ABFE01F19673
:108EA000A8E8B0E082E190E021E08030920719F478
:108EB0000E94006303C0182E0E940063FE01ED5B58
:108EC000FF4FAAE9B0E082E190E021E08030920714
:108ED00019F40E94006303C0182E0E940063FE0173
:108EE000EB5AFF4FADEBB0E082E190E021E0803043
:108EF000920719F40E94006303C0182E0E940063B9
:108F0000CE018D960E949042EAC684E18EA781E050
:108F10008FA78EED88ABFE01F196ACEAB0E080E160
:108F200090E021E08030920719F40E94006303C0B2
:108F3000182E0E940063CE018D960E949042CFC6EB
:108F40000E94392E84E08EA781E08FA781ED88AB47
:108F5000CE018D960E949042C2C688E08EA781E025
:108F60008FA78FED88AB0E94CB2E8BAB0E94CF2EAC
:108F70009AAB89ABFE01ED51FF4FACEBB0E081E065
:108F800090E021E08030920719F40E94006303C052
:108F9000182E0E940063FE01ED51FF4F80818CABC3
:108FA000CE018D960E9490429AC6FE01E358FF4F73
:108FB00080E5DF011D928A95E9F7ACEBB0E081E036
:108FC00090E021E08030920719F40E94116303C001
:108FD000182E0E941163FE01E358FF4FA5E8B0E090
:108FE00081E090E021E08030920719F40E94116343
:108FF00003C0182E0E941163FE01E358FF4FA6E83C
:10900000B0E082E090E021E08030920719F40E9405
:10901000116303C0182E0E94116384E08EA781E0C3
:109020008FA780EE88ABCE018D960E94904257C6E6
:10903000F6018581968190936C0E80936B0E8781EB
:10904000908590936E0E80936D0E8185928590939E
:10905000700E80936F0E83858093710E848580934C
:10906000720E85858093730E878590899093760E16
:109070008093750E86858093740EEBE6FEE0A0E784
:10908000B0E08CE090E021E08030920719F40E947B
:10909000116303C0182E0E94116385E08EA791E032
:1090A0009FA785EA88AB99ABCE018D960E9490422E
:1090B00016C681E18EA781E08FA786EA88AB19AA40
:1090C0008091E200863269F48091E300843049F4B3
:1090D0008091E400833129F484E690E09BAB8AAB75
:1090E00046C08091E2008E3169F48091E3008430C3
:1090F00049F48091E400833129F48DE790E09BAB43
:109100008AAB35C08091E2008E3069F48091E30033
:10911000843049F48091E400833129F48AEF90E0AF
:109120009BAB8AAB24C08091E200863069F48091C9
:10913000E300843049F48091E400833129F484EF22
:1091400091E09BAB8AAB13C08091E200823069F45E
:109150008091E300843049F48091E400833129F464
:1091600088EE93E09BAB8AAB02C01BAA1AAA80913F
:109170006D0E90916E0E9DAB8CAB80916F0E9091A9
:10918000700E9FAB8EAB8091710E88AF8091720E86
:1091900089AF8091730E8AAF8091750E9091760E93
:1091A0009DAF8CAF8091740E8BAFCE018D960E94D7
:1091B000904295C5DE01AB52BF4FF60184818C937E
:1091C0008581FD018183D60116968CE0FE01E9526E
:1091D000FF4F0D9001928A95E1F7FE01ED51FF4F8F
:1091E0001082FE01ED51FF4F8081982F8C30A0F44A
:1091F0009E012B523F4FDF01F901E90FF11D8281E2
:10920000882321F08F3F11F0815082838C918F5FF2
:109210008C93982F8C3080F3CE018B529F4F0E94FD
:10922000D12F84E08EA781E08FA787EA88ABCE019B
:109230008D960E94904253C58E010B521F4FC8015C
:109240000E94EF2F82E18EA781E08FA788EA88AB8A
:10925000D8018C9189ABF80181818AABFE01ED5177
:10926000FF4F1082FE01ED51FF4F8081982F8C300F
:1092700080F49801DF01F901E90FF11D82818F3F30
:1092800011F08F5F82838C918F5F8C93982F8C303D
:1092900090F38CE0DE01A952BF4FFE01F3960D90D2
:1092A00001928A95E1F7CE018D960E94904217C5F2
:1092B000F6018481FE01E358FF4F8083D6011596A5
:1092C0008EE0FE01E258FF4F0D9001928A95E1F782
:1092D000FE01ED51FF4F1082FE01ED51FF4F8081E5
:1092E000982F8E30A0F49E0123583F4FDF01F901E3
:1092F000E90FF11D8181882321F08F3F11F081500A
:1093000081838C918F5F8C93982F8E3080F3DE0158
:10931000A358BF4FF6018389FD018787F601848931
:10932000FD01808BD60155968EE0FE01E257FF4F7E
:109330000D9001928A95E1F7FE01ED51FF4F1082E9
:10934000FE01ED51FF4F8081982F8E30A0F49E01D9
:1093500023583F4FDF01F901E90FF11D818988236F
:1093600021F08F3F11F08150818B8C918F5F8C9316
:10937000982F8E3080F3CE0183589F4F0E94FF2F8D
:1093800084E08EA781E08FA789EA88ABCE018D9615
:109390000E949042A4C48E0103581F4FC8010E942E
:1093A0000F3083E28EA781E08FA78AEA88ABD801CD
:1093B0008C9189ABFE01ED51FF4F1082FE01ED5102
:1093C000FF4F8081982F8E3080F49801DF01F901E2
:1093D000E90FF11D81818F3F11F08F5F81838C91A7
:1093E0008F5F8C93982F8E3090F38EE0DE01A25821
:1093F000BF4FFE01F2960D9001928A95E1F7DE01D2
:10940000A358BF4FFD018785FE01E05CFF4F8083BD
:10941000FD018089FE01EF5BFF4F8083FE01ED516E
:10942000FF4F1082FE01ED51FF4F8081982F8E304B
:1094300080F49D01DF01F901E90FF11D81898F3F62
:1094400011F08F5F818B8C918F5F8C93982F8E3072
:1094500090F38EE0DE01A257BF4FFE01EE5BFF4F9F
:109460000D9001928A95E1F7CE018D960E9490426F
:1094700036C4F601B48085819927982F88272681E4
:10948000820F911DBC018B2D0E94ED2985E08EA7D6
:1094900081E08FA782EC88ABB9AACE018D960E949D
:1094A00090421DC4F601B4808CE08EA781E08FA7A6
:1094B00083EC88ABB9AA8B2D0E94AB298AAB8B2D8C
:1094C0000E94C729892F99278BAB8B2D0E94C72912
:1094D0008CAB8B2D0E94162A892F99278DAB8B2D53
:1094E0000E94162A8EAB8B2D0E942E2A892F992737
:1094F0008FAB8B2D0E942E2A88AFCE018D960E94B5
:109500009042EDC320E0F601848181FD21E0F60167
:10951000848182FD2260F6018181863029F4658193
:10952000822F0E94462ADBC360E0822F0E94462AD7
:10953000D6C30E944B2A84E08EA781E08FA785ECDA
:1095400088ABCE018D960E949042C9C3F601B480CB
:109550009E0123583F4F9581492F4170D9018C912D
:10956000887F9670842B892B8C9386819781F90153
:1095700092838183F60180859185F90194838383A9
:10958000F6018685F9018187F6018785F9018287D1
:10959000F60182859385F90196838583F60184859A
:1095A0009585F90190878783F6018089F901838782
:1095B000F6018189F9018487F6018289F90185879D
:1095C000F6018389F9018687D60154968FE0FE0162
:1095D000E457FF4F0D9001928A95E1F7F60183A1C0
:1095E000F901868FF60184A1F901878FF60185A123
:1095F000F90180A3F60186A1F90181A315E0D60146
:109600009796FE01E156FF4F812F0D9001928A95AA
:10961000E1F7F60184A595A5A6A5B7A5F90187A34D
:1096200090A7A1A7B2A7F60180A9F90183A7B90164
:109630008B2D0E94B13081E08FA782ED88AB1EA7F1
:10964000B9AACE018D960E94904249C3F601B4801A
:109650008E0103581F4FB8018B2D0E94E93081E025
:109660008FA783ED88AB81E38EA7B9AAD8019C911F
:10967000292F21708AA9887F9670822B892B8AAB2B
:10968000F801818192819CAB8BAB838194819EABED
:109690008DAB81858BAF82858CAF8581968198AFAC
:1096A0008FAB878190859AAF89AF83858DAF848595
:1096B0008EAF85858FAF8685FE01E05CFF4F80838E
:1096C0008FE0DE01A457BF4FFE01EF5BFF4F0D900F
:1096D00001928A95E1F7F801868DFE01E05BFF4F6C
:1096E0008083F801878DFE01EF5AFF4F8083F801D8
:1096F00080A1FE01EE5AFF4F8083F80181A1FE0197
:10970000ED5AFF4F808385E0DE01A156BF4FFE0179
:10971000EC5AFF4F0D9001928A95E1F7F80187A16D
:1097200090A5A1A5B2A5FE01E75AFF4F80839183C2
:10973000A283B383F80183A5FE01E35AFF4F808320
:10974000CE018D960E949042CAC2F601B480AE014D
:1097500043585F4F828DDA018C93838DFA018183A8
:10976000F601848DFA018283F6018681FA018383F2
:10977000F6018781FA018483F6018085FA018583E9
:10978000F6018185FA018683F6018285FA018783D5
:10979000F601858DFA01878BC6010B962FE0FE013D
:1097A000EB57FF4FDC010D9001922A95E1F7BA01CA
:1097B0008B2D0E94213181E08FA784ED88AB85E05D
:1097C0008EA7B9AACE018D960E94904288C2F6015A
:1097D000B4808E0103581F4FB8018B2D0E94593160
:1097E00081E08FA785ED88AB8FE18EA7B9AAD8015C
:1097F0008C91FE01E95BFF4F8083F8018181FE01BE
:10980000E85BFF4F8083F8018281FE01E75BFF4F39
:109810008083F80183818BAB84818CAB85818DAB98
:1098200086818EAB87818FAB8789FE01E65BFF4F18
:1098300080838FE0DE01AB57BF4FFE01F8960D909D
:1098400001928A95E1F7CE018D960E94904247C21F
:10985000F6013496AAEEB8E082E090E021E0803094
:10986000920719F40E94116303C0182E0E9411631D
:1098700081E08FA783EE88AB84E08EA7CE018D9622
:109880000E9490422CC281E08FA784EE88AB84E1D5
:109890008EA7FE01F196AAEEB8E082E090E021E00A
:1098A0008030920719F40E94006303C0182E0E94B2
:1098B0000063CE018D960E94904211C2F601B480E1
:1098C000C6010596BC018B2D0E943F3081E08FA719
:1098D00088ED88AB85E08EA7B9AACE018D960E944F
:1098E0009042FDC1F601B48081E08FA789ED88AB7D
:1098F0008EE18EA7B9AABE016E5C7F4F8B2D0E94B0
:109900007830CE018D960E949042E9C1F6018481A3
:109910008093780E85818093790E868180937A0E6C
:10992000878180937B0E808580937C0E81858093D8
:109930007D0E828580937E0E838580937F0EE8E77F
:10994000FEE0AEE6BFE088E090E021E080309207E4
:1099500019F40E94116303C0182E0E94116381E064
:109960008FA785EE88AB84E08EA7CE018D960E94EE
:109970009042B5C181E08FA786EE88AB8CE08EA7C0
:109980008091780E89AB8091790E8AAB80917A0EA6
:109990008BAB80917B0E8CAB80917C0E8DAB8091DC
:1099A0007D0E8EAB80917E0E8FAB80917F0E88AF47
:1099B000CE018D960E94904292C1F6013496AEE897
:1099C000BFE08CE490E021E08030920719F40E941F
:1099D000116303C0182E0E941163F60184818093E5
:1099E000800E8581982F97708091810E887F892BBA
:1099F0008093810E87898093820E808D982F977037
:109A00008091830E887F892B8093830E82A580931B
:109A1000840E83A5982F97708091850E887F892B5F
:109A20008093850E85AD8093860E86AD982F9770B6
:109A30008091870E887F892B8093870E81E08FA786
:109A400087EE88AB84E08EA7CE018D960E9490426F
:109A500046C181E08FA788EE88AB80E58EA7FE0126
:109A6000F196AEE8BFE08CE490E021E08030920710
:109A700019F40E94006303C0182E0E940063CE01F7
:109A80008D960E9490422BC1F6013496AAEDBFE05C
:109A900089E090E021E08030920719F40E94116380
:109AA00003C0182E0E941163F6013D96A3EEBFE09D
:109AB00089E090E021E08030920719F40E94116360
:109AC00003C0182E0E94116381E08FA789EE88AB36
:109AD00084E08EA7CE018D960E94904200C181E065
:109AE0008FA78AEE88AB87E18EA7FE01F196AAEDDB
:109AF000BFE089E090E021E08030920719F40E94F5
:109B0000006303C0182E0E940063FE01FA96A3EEC4
:109B1000BFE089E090E021E08030920719F40E94D4
:109B2000006303C0182E0E940063CE018D960E9430
:109B30009042D5C0C60105960E94B33281E08FA73E
:109B400086ED88AB85E08EA7CE018D960E9490426F
:109B5000C6C081E08FA787ED88AB8DE18EA7CE01CF
:109B6000C2960E94C332CE018D960E949042B7C029
:109B7000F601B480C60104960E94D33281E08FA71B
:109B80008AED88AB85E08EA7B9AACE018D960E949A
:109B90009042A5C0F601B48081E08FA78BED88AB21
:109BA0008AE48EA7BE016F5C7F4F8B2D0E9400332D
:109BB000CE018D960E94904292C0F601B4808B2D0A
:109BC0000E94E41081E08FA78CED88ABB9AA85E0F4
:109BD0008EA7CE018D960E94904281C0F6014481ED
:109BE000558181E08FA78DED88AB86E18EA75AABBA
:109BF00049ABFE01ED51FF4F1082FE01ED51FF4FC9
:109C00008081982F8031C8F48E010F5F1F4FBF01F4
:109C1000892F99279C01200F311F840F951FAA2798
:109C2000BB27ABBFFC018791F90182ABDB018C91B3
:109C30008F5F8C93982F803158F3CE018D960E94C0
:109C400090424DC0F6013496AEE5BFE080E190E071
:109C500021E08030920719F40E94116303C0182E8E
:109C60000E94116381E08FA781EE88AB84E08EA70C
:109C7000CE018D960E94904232C081E08FA782EE85
:109C800088AB84E18EA7FE01F196AEE5BFE080E1EE
:109C900090E021E08030920719F40E94006303C035
:109CA000182E0E940063CE018D960E94904217C02C
:109CB00081E08FA780E888AB85E08EA7F6018381DD
:109CC00089ABCE018D960E94904209C085E08EA797
:109CD0001FA681E088ABCE018D960E949042CD51A7
:109CE000DF4F0FB6F894DEBF0FBECDBFDF91CF912F
:109CF0001F910F91FF90EF90DF90CF90BF90AF90AA
:109D00000895CF93DF93CDB7DEB72A970FB6F894B7
:109D1000DEBF0FBECDBF81E08B8388E88C8384E0FB
:109D20008A83CE0101960E9490422A960FB6F8943B
:109D3000DEBF0FBECDBFDF91CF9108950F931F936C
:109D4000CF93DF93CDB7DEB7C055D0400FB6F894B0
:109D5000DEBF0FBECDBF8A0121E02B832DE52C8312
:109D60009E838D836F8320E0261780F4AE01485FC9
:109D70005F4F822F9927DA01A80FB91FF801E80F6A
:109D8000F91F80818C932F5F261798F38FE08A83C9
:109D9000CE0101960E949042C05BDF4F0FB6F8944F
:109DA000DEBF0FBECDBFDF91CF911F910F91089500
:109DB00048EC50E060E070E083E29BE00E942162AA
:109DC0001092EB0B1092EC0B1092220B0895382F8F
:109DD0002091EC0B83E29BE0FC01E20FF11D30834C
:109DE0008091EC0B8F5F8093EC0B8091220B8F5F47
:109DF0008093220B8091220B883C18F00E94D84E51
:109E000008958091EC0B883C10F01092EC0B0895B3
:109E10009091EC0B8091EB0B981738F08091EC0B44
:109E20009091EB0B891B992708959091EC0B8091F1
:109E3000EB0B981B892F8853992708952091EB0BE2
:109E400083E29BE0FC01E20FF11DE0818091EB0BCE
:109E50008F5F8093EB0B8091220B81508093220BBC
:109E60008091EB0B883C10F01092EB0B8E2F992712
:109E700008950F931F93CF93DF93EC018B0180EC38
:109E80000E94CC50015010408FEF0F3F180709F18E
:109E900088819927803C910521F08B3D910541F007
:109EA0000EC08BED0E94CC508CED0E94CC500AC0AD
:109EB0008BED0E94CC508DED0E94CC5003C0888168
:109EC0000E94CC502196015010408FEF0F3F180791
:109ED000F9F680EC0E94CC50DF91CF911F910F9149
:109EE00008950F931F93382F8091ED0B99270097BA
:109EF00019F00197C1F059C0303C09F056C01092DA
:109F0000EE0B2091EE0B80EF9BE0FC01E20FF11DC8
:109F100030832F5F2093EE0B81E08093ED0B84E67E
:109F20008093EF0B42C0303C99F58091EE0B82306C
:109F3000F0F08091EE0B00EF1BE0F801E80FF11D4F
:109F400030838F5F8093EE0B82E08093ED0B109255
:109F5000EF0BA8016091EE0BC8010E94E04FC80111
:109F60000E94A6421092ED0B1092EE0B1EC01092B2
:109F7000EE0B2091EE0B80EF9BE0FC01E20FF11D58
:109F800030832F5F2093EE0B84E68093EF0B0DC0A0
:109F90002091EE0B80EF9BE0FC01E20FF11D30837E
:109FA0008091EE0B8F5F8093EE0B8091EE0B8936E4
:109FB00020F01092ED0B1092EE0B1F910F9108956F
:109FC000FC01DA0161506F3FF1F02081822F992767
:109FD000803C910521F08B3D910519F010C0319620
:109FE00010C031962081822F99278C3D910521F058
:109FF0008D3D910519F003C020EC01C02BED2D9390
:10A000003196615010F708958091EF0B882389F005
:10A010008091EF0B81508093EF0B9091EF0B992380
:10A0200041F48091ED0B813021F49093EE0B9093ED
:10A03000ED0B089585B1807F85B984B1876084B9BF
:10A0400081E58CBD81E08DBD08958EBD0DB407FE08
:10A05000FDCF8EB5992708950E9489509C9AA498A7
:10A060008FE080935A0CA4986A9862980895A498F7
:10A070000895CF93DF93CDB7DEB728970FB6F89446
:10A08000DEBF0FBECDBFA49B18C0629914C08091E3
:10A09000590C853050F0A4980E94EA1F82E2809308
:10A0A00012011092880E1092770E8091590C8F5FDA
:10A0B0008093590C02C01092590CCE0101960E9457
:10A0C000722929813A8181E590E0289FA001299F8A
:10A0D000500D389F500D1124CA01880F892F881FF9
:10A0E000990B91950E948A508D81882319F48F8154
:10A0F000882311F0A49A01C0A49828960FB6F8946A
:10A10000DEBF0FBECDBFDF91CF91089580935A0C73
:10A1100008950895089510925C0C10925B0C86E0EF
:10A120008093C20088E98093C10060E875E280E016
:10A1300090E00E94A65081E08093F10E1092F20E02
:10A14000089590935C0C80935B0C08959B01AC0187
:10A15000DC01CB01689412F8880F991FAA1FBB1F5E
:10A160001694D1F780509C4DAB40BF4F689413F8C4
:10A17000220F331F441F551F1694D1F7BC01CD0188
:10A180000E948462DA01C9010197292F33272093A5
:10A19000C5008093C4000895982F8091C00085FF6A
:10A1A000FCCF9093C60008950F931F93CF93DF9336
:10A1B0008C01EB0121978FEFCF3FD80751F0F801C9
:10A1C00081918F010E94CC502197FFEFCF3FDF0795
:10A1D000B1F781E090E0DF91CF911F910F91089549
:10A1E0001F920F920FB60F9211242F933F934F930C
:10A1F0005F936F937F938F939F93AF93BF93EF93EF
:10A20000FF938091C6000E94E74EFF91EF91BF91AE
:10A21000AF919F918F917F916F915F914F913F91FE
:10A220002F910F900FBE0F901F901895DC01FB012E
:10A23000415050408FEF4F3F580741F081918D932F
:10A24000415050408FEF4F3F5807C1F70895DC0150
:10A25000FB01415050408FEF4F3F580769F09191FB
:10A260008D91891719F081E090E008954150504098
:10A270008FEF4F3F580799F780E090E00895CF9314
:10A28000DF93DC01FB0160E0462F91E0562F8081D7
:10A29000803231F4692F9F5F319680818032D1F313
:10A2A0008081882379F08081803219F4442309F475
:10A2B000492F8081803209F040E09F5F3196808194
:10A2C000882389F7442331F48081882311F4492FAE
:10A2D00001C0462F262F3327E901C91BD109EC0FF6
:10A2E000FD1F3196842F9927821B930B0197181617
:10A2F000190624F4942F961B915001C090E09150C0
:10A300009F3F29F081918D935F5F9150D8F71C9208
:10A310005F5F852F9927DF91CF910895FC0190E031
:10A320008191882331F09F5F8191882311F09F3FB5
:10A33000D1F7892F99270895DC01FB0180818823BB
:10A3400029F081918D9380818823D9F71C920895FB
:10A350000F931F93CF93DF93082F162FFA0141E03D
:10A36000C0E1D7E2C901BE010E94716261157105A9
:10A3700081F06C9FC0016D9F900D7C9F900D11240A
:10A38000281B390B862F805D8193440F01E015E077
:10A390000AC0153040F0002319F080E3819302C019
:10A3A00080E281934F5FC8EED3E0C901BE010E94F5
:10A3B00071626115710581F06C9FC0016D9F900DF8
:10A3C0007C9F900D1124281B390B862F805D819373
:10A3D0004F5F01E014E00AC0143040F0002319F090
:10A3E00080E3819302C080E281934F5FC4E6D0E0B6
:10A3F000C901BE010E9471626115710581F04F5F54
:10A400006C9FC0016D9F900D7C9F900D1124281BA7
:10A41000390B862F805D819301E013E00AC0133071
:10A4200040F04F5F002319F080E3819302C080E287
:10A430008193C9016AE070E00E9471626115710543
:10A4400091F04F5FCB01880F991F880F991F880FDC
:10A45000991F860F971F860F971F281B390B862F72
:10A46000805D81930AC0123040F04F5F002319F0E5
:10A4700080E3819302C080E28193822F805D81938B
:10A480001082842F9927DF91CF911F910F9108950A
:10A49000FC01262F862F82958F708A3038F06AE073
:10A4A0000E945162892F8F5B819309C0862F82950C
:10A4B0008F706AE00E945162892F805D8193822FA4
:10A4C0008F708A3038F06AE00E945162892F8F5B6A
:10A4D00080830895822F8F706AE00E945162892FD5
:10A4E000805D80830895EF92FF920F931F937C010C
:10A4F0008B01872F9927682FC7010E944852C801F6
:10A500009070682FC7010E9448521F910F91FF90D1
:10A51000EF900895CF92DF92EF92FF920F931F93E7
:10A520006C017A018B01CB01AA27BB27BC01C601B4
:10A530000E947352D801C701A070B070BC01C6015F
:10A540000E9473521F910F91FF90EF90DF90CF9078
:10A5500008951F93CF93DF93CDB7DEB768970FB6FB
:10A56000F894DEBF0FBECDBF10E0BE016F5F7F4F1E
:10A57000812F0E945931412F5527CA01880F991FF9
:10A58000880F991F880F991F9C01241B350BF90117
:10A59000E35AF34F898184838A8185838B81868303
:10A5A0008C8180838D8181838E818283F901E05A41
:10A5B000F34F8F81382F337088858370282F220FB7
:10A5C000220F888D982F9295907F822F832B892B35
:10A5D0008083FA01ED59F24F10821F5F143128F287
:10A5E00068960FB6F894DEBF0FBECDBFDF91CF9156
:10A5F0001F9108951F93CF93DF93CDB7DEB7689770
:10A600000FB6F894DEBF0FBECDBF10E0A89519823B
:10A610001A821B821C821D821E821F821886188E3F
:10A620008FE0189FC00111248858994FBC01CE01BA
:10A6300009960E940062BE016F5F7F4F812F0E94CA
:10A6400021311F5F143110F368960FB6F894DEBF06
:10A650000FBECDBFDF91CF911F910895CF93C0E082
:10A6600086E0C89FC0011124FC01E551F34FF0932F
:10A67000EA0CE093E90C80819181009719F0019731
:10A6800091838083E091E90CF091EA0C82819381BF
:10A69000009719F0019793838283E091E90CF09180
:10A6A000EA0C84819581009719F001979583848342
:10A6B0002C2F3327C901880F991F880F991F880FE6
:10A6C000991F821B930BFC01E35AF34F808188236F
:10A6D00019F48181882321F08C2F8F5D0E947F5493
:10A6E000CF5FC43108F4BCCFCF910895992787304C
:10A6F000910509F466C088309105ACF48430910569
:10A7000009F43EC08530910534F48230910511F191
:10A71000039759F198C08530910509F43CC006971C
:10A7200009F444C090C08A30910509F46BC08B30A5
:10A73000910544F48830910509F44EC0099709F455
:10A7400056C081C08B30910509F467C00C9709F49D
:10A750006FC079C080EC0E942541882319F081E008
:10A7600090E0089580E090E0089581EC0E942541FA
:10A77000882319F081E090E0089580E090E008954A
:10A7800082EC0E942541882319F081E090E0089531
:10A7900080E090E0089581ED0E942541882319F022
:10A7A00081E090E0089580E090E0089584EC0E94BC
:10A7B0002541882319F081E090E0089580E090E041
:10A7C000089585EC0E942541882319F081E090E0EE
:10A7D000089580E090E0089586EC0E94254188234A
:10A7E00019F081E090E0089580E090E0089587EC12
:10A7F0000E942541882319F081E090E0089580E0CF
:10A8000090E0089583EC0E942541882319F081E0AF
:10A8100090E0089580E090E0089582ED0E94254147
:10A82000882319F081E090E0089580E090E0089599
:10A8300083ED0E942541882319F081E090E008957E
:10A8400080E090E0089580E090E008950F93CF932A
:10A85000DF93CDB7DEB721970FB6F894DEBF0FBEFA
:10A86000CDBF89838150843170F000E021E0AE01DA
:10A870004F5F5F4F69E071E08FE891E00E94B42C78
:10A8800080E090E007C089819927FC01EE59F24FE2
:10A890008081992721960FB6F894DEBF0FBECDBFF9
:10A8A000DF91CF910F9108950F93CF93DF93CDB7A1
:10A8B000DEB721970FB6F894DEBF0FBECDBF8983F8
:10A8C000843160F000E021E0AE014F5F5F4F64E152
:10A8D00071E08FE891E00E94B42C07C0898123E6E3
:10A8E0003DE0F901E80FF11D608321960FB6F89461
:10A8F000DEBF0FBECDBFDF91CF910F910895FF92C4
:10A900000F931F93CF93DF93CDB7DEB721970FB689
:10A91000F894DEBF0FBECDBF1982813209F46DC03D
:10A92000823219F481E0898368C0833219F482E0AD
:10A93000898363C0843219F483E089835EC08532E1
:10A9400019F484E0898359C0863219F485E089833B
:10A9500054C0873219F486E089834FC0883219F4D5
:10A9600087E089834AC0893219F488E0898345C029
:10A970008A3219F489E0898340C08B3219F48AE065
:10A9800089833BC08C3219F48BE0898336C08D32C9
:10A9900019F48CE0898331C08E3219F48DE08983FB
:10A9A0002CC08F3219F48EE0898327C0803319F4CC
:10A9B0008FE0898322C0813319F480E189831DC02F
:10A9C000823319F481E1898318C0833319F482E159
:10A9D000898313C0843319F483E189830EC000E0B6
:10A9E00021E0AE014F5F5F4F69E471E08FE891E0D5
:10A9F0000E94B42C80E090E087C700E0102FF02E7A
:10AA0000298186E0289FC00111248551934F90939E
:10AA1000EA0C8093E90C3327C901880F991F880F2E
:10AA2000991F880F991F821B930BFC01E35AF34F68
:10AA30008081882309F49BC18981282F3327C9018C
:10AA4000880F991F880F991F880F991F821B930BDE
:10AA5000FC01E35AF34F80818F3F11F411E087C16D
:10AA60008981282F3327C901880F991F880F991FC3
:10AA7000880F991F821B930BFC01E35AF34FE0816F
:10AA80008E2F82508B3008F04DC08E2F0E9476534F
:10AA9000482F8981282F3327C901880F991F880FD4
:10AAA000991F880F991F821B930BFC01E05AF34FEB
:10AAB000808182958F7080FF02C081E04827442307
:10AAC00061F0E091E90CF091EA0C80819181892B91
:10AAD00011F411E04CC110E04AC1A091E90CB09111
:10AAE000EA0C8981282F3327C901880F991F880F05
:10AAF000991F880F991F821B930BFC01E35AF34F98
:10AB0000948185E0989FC00111248D939C93E091DE
:10AB1000E90CF091EA0C8081918101969183808308
:10AB200010E025C18981282F3327C901880F991F7B
:10AB3000880F991F880F991F821B930BFC01E35A02
:10AB4000F34FE0818E2F8D50803208F04DC08F5F23
:10AB50000E94E710482F8981282F3327C901880FC9
:10AB6000991F880F991F880F991F821B930BFC0157
:10AB7000E05AF34F808182958F7080FF02C081E0A0
:10AB80004827442361F0E091E90CF091EA0C8081C0
:10AB90009181892B11F411E0EAC010E0E8C0A09186
:10ABA000E90CB091EA0C8981282F3327C901880F5D
:10ABB000991F880F991F880F991F821B930BFC0107
:10ABC000E35AF34F948185E0989FC00111248D933F
:10ABD0009C93E091E90CF091EA0C808191810196BF
:10ABE0009183808310E0C3C08981282F3327C90156
:10ABF000880F991F880F991F880F991F821B930B2D
:10AC0000FC01E35AF34FE0818E2F8D52823208F01F
:10AC10004DC08F5F0E942C29482F8981282F332710
:10AC2000C901880F991F880F991F880F991F821BD0
:10AC3000930BFC01E05AF34F808182958F7080FF67
:10AC400002C081E04827442361F0E091E90CF091D3
:10AC5000EA0C80819181892B11F411E088C010E009
:10AC600086C0A091E90CB091EA0C8981282F332786
:10AC7000C901880F991F880F991F880F991F821B80
:10AC8000930BFC01E35AF34F948185E0989FC00138
:10AC900011248D939C93E091E90CF091EA0C808152
:10ACA000918101969183808310E061C08981282F72
:10ACB0003327C901880F991F880F991F880F991F83
:10ACC000821B930BFC01E35AF34FE0818E2F8F54CC
:10ACD0008F3008F04CC08F5F0E942654482F898126
:10ACE000282F3327C901880F991F880F991F880FB4
:10ACF000991F821B930BFC01E05AF34F80818295D0
:10AD00008F7080FF02C081E04827442361F0E0910A
:10AD1000E90CF091EA0C80819181892B11F411E00A
:10AD200026C010E024C0A091E90CB091EA0C898102
:10AD3000282F3327C901880F991F880F991F880F63
:10AD4000991F821B930BFC01E35AF34F948185E01A
:10AD5000989FC00111248D939C93E091E90CF09190
:10AD6000EA0C8081918101969183808310E0898132
:10AD7000282F3327C901880F991F880F991F880F23
:10AD8000991F821B930BFC01E35AF34F81818823A7
:10AD900011F4082F9FC18981282F3327C901880FFB
:10ADA000991F880F991F880F991F821B930BFC0115
:10ADB000E35AF34F81818F3F11F401E08BC1898108
:10ADC000282F3327C901880F991F880F991F880FD3
:10ADD000991F821B930BFC01E35AF34F9181892F3A
:10ADE00082508B3008F04EC0892F0E947653482F36
:10ADF0008981282F3327C901880F991F880F991F30
:10AE0000880F991F821B930BFC01E05AF34F80813E
:10AE100082958F7081FF02C081E04827442361F052
:10AE2000E091E90CF091EA0C82819381892B11F475
:10AE300001E050C100E04EC1A091E90CB091EA0CD4
:10AE40008981282F3327C901880F991F880F991FDF
:10AE5000880F991F821B930BFC01E35AF34F9581D6
:10AE600085E0989FC0011124FD0193838283E091C6
:10AE7000E90CF091EA0C828193810196938382839D
:10AE800000E028C18981282F3327C901880F991F25
:10AE9000880F991F880F991F821B930BFC01E35A9F
:10AEA000F34F9181892F8D50803208F04EC08F5F13
:10AEB0000E94E710482F8981282F3327C901880F66
:10AEC000991F880F991F880F991F821B930BFC01F4
:10AED000E05AF34F808182958F7081FF02C081E03C
:10AEE0004827442361F0E091E90CF091EA0C82815B
:10AEF0009381892B11F401E0EDC000E0EBC0A0913B
:10AF0000E90CB091EA0C8981282F3327C901880FF9
:10AF1000991F880F991F880F991F821B930BFC01A3
:10AF2000E35AF34F958185E0989FC0011124FD01FC
:10AF300093838283E091E90CF091EA0C8281938102
:10AF400001969383828300E0C5C08981282F33272F
:10AF5000C901880F991F880F991F880F991F821B9D
:10AF6000930BFC01E35AF34F9181892F8D5282326A
:10AF700008F04EC08F5F0E942C29482F8981282F0E
:10AF80003327C901880F991F880F991F880F991FB0
:10AF9000821B930BFC01E05AF34F808182958F70E6
:10AFA00081FF02C081E04827442361F0E091E90C71
:10AFB000F091EA0C82819381892B11F401E08AC01F
:10AFC00000E088C0A091E90CB091EA0C8981282F9B
:10AFD0003327C901880F991F880F991F880F991F60
:10AFE000821B930BFC01E35AF34F958185E0989FF8
:10AFF000C0011124FD0193838283E091E90CF0915B
:10B00000EA0C8281938101969383828300E062C07F
:10B010008981282F3327C901880F991F880F991F0D
:10B02000880F991F821B930BFC01E35AF34F918108
:10B03000892F8F548F3008F04DC08F5F0E942654A7
:10B04000482F8981282F3327C901880F991F880F1E
:10B05000991F880F991F821B930BFC01E05AF34F35
:10B06000808182958F7081FF02C081E04827442350
:10B0700061F0E091E90CF091EA0C82819381892BD7
:10B0800011F401E027C000E025C0A091E90CB091C7
:10B09000EA0C8981282F3327C901880F991F880F4F
:10B0A000991F880F991F821B930BFC01E35AF34FE2
:10B0B000958185E0989FC0011124FD0193838283CF
:10B0C000E091E90CF091EA0C8281938101969383DF
:10B0D000828300E08981282F3327C901880F991FB7
:10B0E000880F991F880F991F821B930BFC01E35A4D
:10B0F000F34F8281882311F4F82EA4C18981282F6F
:10B100003327C901880F991F880F991F880F991F2E
:10B11000821B930BFC01E35AF34F82818F3F19F49A
:10B12000FF24F3948FC18981282F3327C901880F09
:10B13000991F880F991F880F991F821B930BFC0181
:10B14000E35AF34F9281892F82508B3008F04FC021
:10B15000892F0E947653482F8981282F3327C901D0
:10B16000880F991F880F991F880F991F821B930BB7
:10B17000FC01E05AF34F808182958F7082FF02C0FC
:10B1800081E04827442369F0E091E90CF091EA0C52
:10B1900084819581892B19F4FF24F39453C1FF24F2
:10B1A00051C1A091E90CB091EA0C8981282F332775
:10B1B000C901880F991F880F991F880F991F821B3B
:10B1C000930BFC01E35AF34F968185E0989FC001F1
:10B1D0001124FD0195838483E091E90CF091EA0C40
:10B1E00084819581019695838483FF242BC1898175
:10B1F000282F3327C901880F991F880F991F880F9F
:10B20000991F821B930BFC01E35AF34F9281892F04
:10B210008D50803208F04FC08F5F0E94E710482F9A
:10B220008981282F3327C901880F991F880F991FFB
:10B23000880F991F821B930BFC01E05AF34F80810A
:10B2400082958F7082FF02C081E04827442369F015
:10B25000E091E90CF091EA0C84819581892B19F435
:10B26000FF24F394EFC0FF24EDC0A091E90CB0914E
:10B27000EA0C8981282F3327C901880F991F880F6D
:10B28000991F880F991F821B930BFC01E35AF34F00
:10B29000968185E0989FC0011124FD0195838483E8
:10B2A000E091E90CF091EA0C8481958101969583F7
:10B2B0008483FF24C7C08981282F3327C901880FC1
:10B2C000991F880F991F880F991F821B930BFC01F0
:10B2D000E35AF34F9281892F8D52823208F04FC08A
:10B2E0008F5F0E942C29482F8981282F3327C9017D
:10B2F000880F991F880F991F880F991F821B930B26
:10B30000FC01E05AF34F808182958F7082FF02C06A
:10B3100081E04827442369F0E091E90CF091EA0CC0
:10B3200084819581892B19F4FF24F3948BC0FF2429
:10B3300089C0A091E90CB091EA0C8981282F3327AC
:10B34000C901880F991F880F991F880F991F821BA9
:10B35000930BFC01E35AF34F968185E0989FC0015F
:10B360001124FD0195838483E091E90CF091EA0CAE
:10B3700084819581019695838483FF2463C08981AC
:10B38000282F3327C901880F991F880F991F880F0D
:10B39000991F821B930BFC01E35AF34F9281892F73
:10B3A0008F548F3008F04EC08F5F0E942654482F74
:10B3B0008981282F3327C901880F991F880F991F6A
:10B3C000880F991F821B930BFC01E05AF34F808179
:10B3D00082958F7082FF02C081E04827442369F084
:10B3E000E091E90CF091EA0C84819581892B19F4A4
:10B3F000FF24F39427C0FF2425C0A091E90CB0914D
:10B40000EA0C8981282F3327C901880F991F880FDB
:10B41000991F880F991F821B930BFC01E35AF34F6E
:10B42000968185E0989FC0011124FD019583848356
:10B43000E091E90CF091EA0C848195810196958365
:10B440008483FF242981822F9927AC01440F551F43
:10B45000440F551F440F551F481B590BDA01A35ABF
:10B46000B34F8C91882309F47FC1FD01818188232A
:10B4700009F47AC18281882309F476C1FA01E05A7D
:10B48000F34FE0818E2F837009F084C0112309F4FB
:10B490003EC00023E1F18E2F86958695837061F47E
:10B4A0006F2D822F0E945454FF2019F081E090E00C
:10B4B0002BC280E090E028C28981282F3327C90160
:10B4C000880F991F880F991F880F991F821B930B54
:10B4D000FC01E05AF34F8081869586958370823017
:10B4E00079F460E01F1509F461E089810E945454E9
:10B4F0001F1519F481E090E007C280E090E004C2DB
:10B5000061E089810E94545481E090E0FDC149814D
:10B51000242F3327C901880F991F880F991F880F7F
:10B52000991F821B930BFC01E05AF34F8081869593
:10B5300086958370823049F4FF2039F461E0842FCE
:10B540000E94545481E090E0DFC14981242F3327C9
:10B55000C901880F991F880F991F880F991F821B97
:10B56000930BFC01E05AF34F808186958695682FF6
:10B570006370613041F4FF2031F0842F0E945454F5
:10B5800081E090E0C1C160E089810E94545480E074
:10B5900090E0BAC14981242F3327C901880F991F30
:10B5A000880F991F880F991F821B930BFC01E05A8B
:10B5B000F34FE0818E2F8370823009F045C0101761
:10B5C000E1F58E2F86958695837061F46F2D842F1B
:10B5D0000E945454FF2019F081E090E095C180E072
:10B5E00090E092C18981282F3327C901880F991FC4
:10B5F000880F991F880F991F821B930BFC01E05A3B
:10B60000F34F8081869586958370823079F460E06F
:10B610001F1509F461E089810E9454541F1519F423
:10B6200081E090E071C180E090E06EC161E08981CD
:10B630000E94545481E090E067C160E089810E94DB
:10B64000545480E090E060C1112319F4002309F400
:10B6500048C04981242F3327C901880F991F880FBB
:10B66000991F880F991F821B930BFC01E05AF34F1F
:10B67000808186958695837061F46F2D842F0E945A
:10B680005454FF2019F081E090E03EC180E090E04A
:10B690003BC14981242F3327C901880F991F880F87
:10B6A000991F880F991F821B930BFC01E05AF34FDF
:10B6B0008081869586958370823061F46F2D842F0A
:10B6C0000E945454FF2019F081E090E01DC180E0F9
:10B6D00090E01AC161E089810E94545481E090E0B9
:10B6E00013C14981242F3327C901880F991F880F5F
:10B6F000991F880F991F821B930BFC01E05AF34F8F
:10B70000808186958695682F6370613041F4FF20B3
:10B7100021F1842F0E94545481E090E0F5C04981CA
:10B72000242F3327C901880F991F880F991F880F6D
:10B73000991F821B930BFC01E05AF34F8081869581
:10B7400086958370823049F4FF2039F461E0842FBC
:10B750000E94545481E090E0D7C060E089810E944B
:10B76000545480E090E0D0C02981822F9927AC0109
:10B77000440F551F440F551F440F551F481B590BAD
:10B78000DA01A35AB34F8C91882309F452C0FD010A
:10B790008181882309F44DC0FA01E05AF34F80817A
:10B7A000837091F4112349F0002339F061E0822F76
:10B7B0000E94545481E090E0A7C060E089810E941B
:10B7C000545480E090E0A0C04981242F3327C90160
:10B7D000880F991F880F991F880F991F821B930B41
:10B7E000FC01E05AF34F80818370823081F410179E
:10B7F00039F461E0842F0E94545481E090E084C0C9
:10B8000060E089810E94545480E090E07DC0112363
:10B8100011F4002339F061E089810E94545481E0E1
:10B8200090E072C060E089810E94545480E090E012
:10B830006BC02981822F9927AC01440F551F440FFB
:10B84000551F440F551F481B590BDA01A35AB34F1C
:10B85000FD018181882309F455C08281882309F480
:10B8600051C0FA01E05AF34F808186958695837026
:10B8700091F4112349F0002339F061E0822F0E94F6
:10B88000545481E090E040C060E089810E945454AB
:10B8900080E090E039C04981242F3327C901880F07
:10B8A000991F880F991F880F991F821B930BFC010A
:10B8B000E05AF34F8081869586958370823081F4BB
:10B8C000101739F461E0842F0E94545481E090E015
:10B8D0001BC060E089810E94545480E090E014C055
:10B8E000112311F4002339F061E089810E9454543E
:10B8F00081E090E009C060E089810E94545480E0BA
:10B9000090E002C080E090E021960FB6F894DEBF90
:10B910000FBECDBFDF91CF911F910F91FF90089582
:10B92000CF93DF93CDB7DEB721970FB6F894DEBF84
:10B930000FBECDBF282F04B603FE28C0FE013196EE
:10B94000ACEBB0E081E090E031E08030930719F497
:10B950000E94006303C0182E0E9400638981843115
:10B9600090F48F5F8983FE013196ACEBB0E081E00B
:10B9700090E031E08030930719F40E94116303C016
:10B98000182E0E94116384B7877F84BF8091600066
:10B9900088618093600020936000809160008860DF
:10B9A0008093600021960FB6F894DEBF0FBECDBF26
:10B9B000DF91CF910895EF92FF920F931F937B0138
:10B9C0008C0120E030E040E05FE40E943F5F88238C
:10B9D0009CF020E030E040E05FECC801B7010E943D
:10B9E000295EDC01CB01BC01CD010E94D95F605012
:10B9F00070408040904804C0C801B7010E94D95FE0
:10BA00001F910F91FF90EF900895A0E0B0E0EBE060
:10BA1000FDE50C94C1628C017B015A01DC018C9123
:10BA2000823058F0FB019081923010F4A7010BC1D5
:10BA3000843029F4943009F4A6C0A80104C19430DC
:10BA4000A9F3923009F4A9C0823081F3F801C280D1
:10BA5000D380FB0162817381F801248135814681A5
:10BA60005781F7016480758086809780C601861BA8
:10BA7000970B97FDD8C080970CF46CC06C157D05B2
:10BA80000CF0ADC0662477244301F8016181F70111
:10BA90008181681709F499C0662309F491C0621A7C
:10BAA000730A840A950AA401930157FDC0C0F501E9
:10BAB0001182B60119012A0179018A0139014A016D
:10BAC00008946108710881089108FFEF6F16FFEF75
:10BAD0007F06FFEF8F06FFE39F06F0F4A8019701B2
:10BAE000220F331F441F551F19012A01B60161504F
:10BAF00070406B0179018A0139014A01089461089B
:10BB00007108810891088FEF68168FEF78068FEF24
:10BB100088068FE3980610F383E0D5018C9357FCD9
:10BB200064C0F5012483358346835783738362831E
:10BB3000A50189C06F5F7F4FD401C30181709070F0
:10BB4000A070B0709694879477946794682A792A45
:10BB50008A2A9B2A6C157D056CF311C00894C11CC0
:10BB6000D11CDA01C90181709070A070B070569537
:10BB7000479537952795282B392B4A2B5B2BC616D3
:10BB8000D70664F382CFF8019181FB018181981778
:10BB900009F453CF42EA51E056C0823009F04DCF4C
:10BBA00088E0DA01F80101900D928A95E1F7F80139
:10BBB0008181FB0191818923FA018183A50143C021
:10BBC000261937094809590970CFF5016183B60173
:10BBD000260D371D481D591D19012A019DCF6B01E6
:10BBE00020E030E040E050E050CFD201C101B695F6
:10BBF000A7959795879521E030E040E050E022221C
:10BC0000332244225522282A392A4A2A5B2AF5015E
:10BC100024823582468257820894C11CD11CD3826B
:10BC2000C282A50110C0909581959F4F24CF81E0DD
:10BC3000F5018183B60150954095309521953F4F90
:10BC40004F4F5F4F37CFCA01E2E1CDB7DEB70C945B
:10BC5000DD62A0E2B0E0EFE2FEE50C94CF62DC0131
:10BC6000CB01898F9A8FAB8FBC8F2D8F3E8F4F8FDB
:10BC700058A3BE016F5F7F4FCE0149960E941361AA
:10BC80008E01075F1F4FB801CE014D960E941361D0
:10BC9000AE014F5E5F4FB801CE0101960E94055D77
:10BCA0000E942B60DC01CB01BC01CD01E4E0A09639
:10BCB0000C94EB62A0E2B0E0E0E6FEE50C94CF620B
:10BCC000DC01CB01898F9A8FAB8FBC8F2D8F3E8F7C
:10BCD0004F8F58A3BE016F5F7F4FCE0149960E94E0
:10BCE00013618E01075F1F4FB801CE014D960E9470
:10BCF00013618A8591E089278A87AE014F5E5F4F85
:10BD0000B801CE0101960E94055D0E942B60DC0106
:10BD1000CB01BC01CD01E4E0A0960C94EB62A8E15C
:10BD2000B0E0E5E9FEE50C94C962DC01CB01898B4A
:10BD30009A8BAB8BBC8B2D8B3E8B4F8B588FBE0160
:10BD40006F5F7F4FCE0141960E9413618E01075FA6
:10BD50001F4FB801CE0145960E941361FE01319636
:10BD60002981223008F45FC03985323010F4B801DF
:10BD70007BC081819A8589278183243009F455C04D
:10BD8000223009F452C0343009F454C0323009F47E
:10BD900058C06B817C818B859C85681B790B2D81BC
:10BDA0003E814F815885ED84FE840F8518892E15BC
:10BDB0003F054007510730F4220F331F441F551F22
:10BDC000615070407C836B8380E090E0A0E0B0E441
:10BDD000AA24BB2465012E153F054007510740F0FA
:10BDE000A82AB92ACA2ADB2A2E193F09400B510B6F
:10BDF000B695A79597958795220F331F441F551F1A
:10BE00000097A105B10539F7D601C5018F7790706C
:10BE1000A070B07080349105A105B105A9F0A4828D
:10BE2000B582C682D782BF011FC02317E1F762EA3D
:10BE300071E01AC01D821E821F8218861C821B821E
:10BE4000F2CF84E08983EFCFA7FC05C0211531052F
:10BE50004105510521F380E490E0A0E0B0E0A80E98
:10BE6000B91ECA1EDB1EDBCFCB010E942B60DC019A
:10BE7000CB01BC01CD01EAE068960C94E562A8E133
:10BE8000B0E0E5E4FFE50C94CF62DC01CB01898BE7
:10BE90009A8BAB8BBC8B2D8B3E8B4F8B588FBE01FF
:10BEA0006F5F7F4FCE0141960E9413618E01075F45
:10BEB0001F4FB801CE0145960E94136189818230DF
:10BEC00018F08985823018F42FEF3FEF09C0B801D0
:10BED000CE0101960E948D61282F332727FD3095D2
:10BEE000C901E4E068960C94EB62A8E0B0E0EBE7EF
:10BEF000FFE50C94CD629B01AC017B018C01EE242B
:10BF000017FDE394FF2400271127EA82211531054C
:10BF10004105510539F482E08983CE0101960E94E2
:10BF20002B6043C083E089836EE170E0CB01EE209B
:10BF300031F579018A01A80197012030E0E03E0740
:10BF4000E0E04E07E0E45E0798F479018A01EE0C28
:10BF5000FF1C001F111F0197BC01A8019701E0E021
:10BF6000EE16E0E0FE06E0E00E07E0E41E0768F3F0
:10BF7000ED82FE820F8318877C836B83CECF2030C7
:10BF8000E0E03E07E0E04E07E0E85E0741F0EE2427
:10BF9000FF248701E21AF30A040B150BCCCF7C8334
:10BFA0006B8360E070E080E09FECE6E028960C9404
:10BFB000E962ACE0B0E0EFEDFFE50C94D162DC01AA
:10BFC000CB0189879A87AB87BC87BE016F5F7F4FA4
:10BFD000CE0109960E9413618981823011F082306E
:10BFE00028F460E070E080E090E031C0843039F007
:10BFF0002B813C8137FDF5CF2F3131056CF08A81E3
:10C00000882329F060E070E080E090E820C06FEFC6
:10C010007FEF8FEF9FE71BC08EE190E0821B930BB9
:10C020002D813E814F81588504C05695479537959F
:10C0300027958A95D2F78A81882339F050954095C3
:10C04000309521953F4F4F4F5F4FCA01B901E2E054
:10C050002C960C94ED62A0E0B0E0E1E3F0E60C94E5
:10C06000C762882499245401DC01FC0124813581B4
:10C07000468157818181082F112760E070E08C9103
:10C08000823020F46FEF70E04061A4C0843009F486
:10C0900064C0823009F463C02115310541055105A2
:10C0A00009F498C0FD0182819381FFEF82389F07D8
:10C0B0000CF050C0A2E8EA2EAFEFFA2EE81AF90A07
:10C0C0008AE1E816F1040CF06BC06B0181E090E0AE
:10C0D000A0E0B0E00E2C04C0880F991FAA1FBB1F60
:10C0E0000A94D2F70197A109B10982239323A423CB
:10C0F000B5230097A105B10519F0F1E0CF2ED12CA1
:10C1000004C05695479537952795EA94D2F7C6010E
:10C11000AA2797FDA095BA2F282B392B4A2B5B2BEA
:10C12000DA01C9018F779070A070B07080349105EA
:10C13000A105B105D1F1215C3F4F4F4F5F4F20303A
:10C14000E0E03E07E0E04E07E0E45E0708F161E072
:10C1500070E01EC0803891053CF06FEF70E020E089
:10C1600030E040E050E036C0BC0161587F4FDA015A
:10C17000C9018F779070A070B07080349105A105CF
:10C18000B105D1F0215C3F4F4F4F5F4F57FD1BC0B2
:10C1900097E056954795379527959A95D1F71AC008
:10C1A00020E030E040E050E0BBCF27FFC8CF205C6C
:10C1B0003F4F4F4F5F4FC3CF27FFE8CF205C3F4F2C
:10C1C0004F4F5F4FE3CF56954795379527956F5F54
:10C1D0007F4FDECF822E932E942F9F778A2D8078EB
:10C1E000A82EA92A962F9795992797958A2D8F770C
:10C1F000A82EA92A76956795962F9F778B2D807804
:10C20000B82EB92A902F9795992797958B2D8F77D0
:10C21000B82EB92AD501C401BC01CD01ECE0CDB7DF
:10C22000DEB70C94E362CF93DF93FC01DB01408126
:10C2300051812281622F6F7770E0221F2227221FF7
:10C240009381892F880F822B282F3327991F9927B5
:10C25000991FED0199832115310541F441155105CF
:10C2600061057105E1F482E08C9354C02F3F3105E4
:10C2700009F441C02F573040FD013383228383E00E
:10C280008C9387E0440F551F661F771F8A95D1F75F
:10C290007064ED014C835D836E837F833BC022E835
:10C2A0003FEFF901C7E0440F551F661F771FCA957E
:10C2B000D1F783E08C93403080E0580780E0680736
:10C2C00080E4780778F4440F551F661F771F2150CC
:10C2D0003040F9014030C0E05C07C0E06C07C0E4CA
:10C2E0007C0788F3ED01FB83EA83FD0144835583DA
:10C2F000668377830FC0411551056105710519F4F7
:10C3000084E08C9307C064FF03C081E08C93C1CFAD
:10C310001C92BFCFDF91CF9108950F931F93CF93BE
:10C32000DF93FC01DB018081823018F09C91923018
:10C3300018F461E070E05EC08430C1F0843001F137
:10C34000943009F447C0823009F44BC0823009F4BC
:10C350004EC09230A9F04181ED0189814817B9F0B2
:10C36000442389F08FEF9FEFBC0144C0943031F734
:10C37000EB018981682F77278181681B71093AC099
:10C380008181882379F781E090E0BC0133C022816C
:10C390003381ED018A819B81821793070CF3281763
:10C3A00039079CF00481158126813781FD01648164
:10C3B000758186819781601771078207930780F2E4
:10C3C000061717072807390778F4442359F281E044
:10C3D00090E0DBCFFD018181882321F281E090E0B4
:10C3E000D4CF923009F0B2CF60E070E003C0ED012D
:10C3F0008981F2CFCB01DF91CF911F910F910895E9
:10C40000FB01DC0105900D920020E1F70895FB018E
:10C41000DC0104C08D910190801921F441505040FD
:10C42000C8F7881B990B0895FB01DC0140FF05C08C
:10C4300002C001900D9201900D9242505040C8F7F9
:10C440000895DC0140FF03C001C06D936D9342501D
:10C450005040D8F70895FB01DC0101900D920020B7
:10C46000E1F70895629FD001739FF001829FE00D74
:10C47000F11D649FE00DF11D929FF00D839FF00D63
:10C48000749FF00D659FF00D9927729FB00DE11D0F
:10C49000F91F639FB00DE11DF91FBD01CF011124EC
:10C4A0000895991B79E004C0991F961708F0961B10
:10C4B000881F7A95C9F780950895AA1BBB1B51E187
:10C4C00007C0AA1FBB1FA617B70710F0A61BB70B04
:10C4D000881F991F5A95A9F780959095BC01CD01A9
:10C4E000089597FB092E07260AD077FD04D0E5DFD3
:10C4F00006D000201AF4709561957F4F0895F6F7E5
:10C50000909581959F4F0895A1E21A2EAA1BBB1BFF
:10C51000FD010DC0AA1FBB1FEE1FFF1FA217B3070F
:10C52000E407F50720F0A21BB30BE40BF50B661F25
:10C53000771F881F991F1A9469F7609570958095E9
:10C5400090959B01AC01BD01CF01089597FB092E89
:10C5500005260ED057FD04D0D7DF0AD0001C38F4D2
:10C5600050954095309521953F4F4F4F5F4F08951F
:10C57000F6F790958095709561957F4F8F4F9F4FFF
:10C5800008952F923F924F925F926F927F928F9277
:10C590009F92AF92BF92CF92DF92EF92FF920F9352
:10C5A0001F93CF93DF93CDB7DEB7CA1BDB0B0FB65C
:10C5B000F894DEBF0FBECDBF09942A883988488819
:10C5C0005F846E847D848C849B84AA84B984C884AF
:10C5D000DF80EE80FD800C811B81AA81B981CE0FA6
:10C5E000D11D0FB6F894DEBF0FBECDBFED0108958B
:10C5F000F999FECFB2BDA1BDF89A119600B4089585
:10C60000F7DF01921A94E1F70895F999FECFB2BDD0
:10C61000A1BD00BC11960FB6F894FA9AF99A0FBE14
:0CC6200008950190F2DF1A94E1F70895EC
:10C62C0001012E2E2F63616E5F696E7075742E631F
:10C63C00006E222E2E2F6368616E6E656C732E63F6
:10C64C000053657175656E63652023310053657108
:10C65C0075656E63652023320053657175656E6375
:10C66C00652023330053657175656E636520233433
:10C67C0000455233002E2E2F656570726F6D636806
:10C68C00616E6E656C732E630050434D30004552E5
:10C69C0033004C4F4730340050434D2076657220A8
:10C6AC00392E3132004F425220383434300B002EA8
:10C6BC002E2F7669727475656C5F696E7075742E49
:0AC6CC006300000000000000000001
:00000001FF
